:020000040000FA
:1000000002EF00F00F013F0E926E000E936E000E95
:10001000946E030E956E0F0E966E000E386F000EE6
:10002000396F000E3A6F000E3B6F000E3C6F806A16
:10003000816A826A836A846A896A8A6A8B6A8C6A3C
:100040008D6A00018B8C006A016A026A036A046A85
:10005000056A066A076A086A096A0A6A0B6A0C6A0C
:100060000D6A0E6A0F6A106A116A126A136A146ABC
:10007000156A166A176A186A196A1A6A1B6A1C6A6C
:100080001D6A1E6A1F6A206A216A226A236A256A1B
:10009000266A276A296A246A286A2A6A2B6A2C6ACD
:1000A0002D6A2E6A2F6A306A316A326A336A346A7C
:1000B000356A366A376A386A396A3A6A3C6A3B6A2C
:1000C0003D6A3E6A3F6A406A416A426A436A446ADC
:1000D000456A466A476A486A496A4A6A4B6A4C6A8C
:1000E0004D6A4E6A506A516A526AD3EC35F0D3ECCD
:1000F00035F0D3EC35F0D3EC35F020EC2AF0C00E1F
:100100008A6E8C9C8C9E8C8A8C9A1FEC2BF03F0EF6
:100110008A6E8C9C8C9E8C8A8C9A42EC2BF08B8AFB
:1001200023EC2AF0FBEC35F0000EAA6E000EA96E4F
:10013000A69EA69CA68000000000A850116E000E8E
:10014000AA6E010EA96EA69EA69CA68000000000C5
:10015000A850126E000EAA6E020EA96EA69EA69C54
:10016000A68000000000A850136E000EAA6E030EB9
:10017000A96EA69EA69CA68000000000A850146E42
:10018000000EAA6E040EA96EA69EA69CA680000074
:100190000000A850156E000EAA6E050EA96EA69E50
:1001A000A69CA68000000000A850166E000EAA6E45
:1001B000060EA96EA69EA69CA68000000000A85070
:1001C000176E000EAA6E070EA96EA69EA69CA680AC
:1001D00000000000A850186E000EAA6E080EA96E4E
:1001E000A69EA69CA68000000000A850196E000ED6
:1001F000AA6E090EA96EA69EA69CA680000000000D
:10020000A8501A6E000EAA6E0A0EA96EA69EA69C93
:10021000A68000000000A8504C6E5FEC2BF0A4EC10
:100220002CF01D504E6E4CA41BEF01F083A21BEF6F
:1002300001F0AEEC34F0A4EC2CF080B280B63FEFCD
:1002400001F03EB640EF01F01550380B406E380E0D
:10025000405CD8B430EF01F0080E402632EF01F0D8
:10026000000E406E1550C70B156E405015124CB263
:10027000CBEC34F05FEC2BF03E8640EF01F03E9685
:1002800080B461EF01F03EB462EF01F01550380B1D
:10029000406E000E405CD8B452EF01F0080E405E94
:1002A00054EF01F0380E406E1550C70B156E4050DC
:1002B00015124CB2CBEC34F05FEC2BF03E8462EFC5
:1002C00001F03E944CB4A9EC34F080B279EF01F027
:1002D0003EB27AEF01F0040E415CD8B473EF01F046
:1002E000412A74EF01F0416A42EC2BF03E827AEF32
:1002F00001F03E92000E415CD8B495EF01F0010E82
:10030000415CD8B48AEF0BF0020E415CD8B4ACEF7C
:1003100011F0030E415CD8B48AEF20F0040E415C6A
:10032000D8B405EF26F01BEF01F01AEC2AF0410ECD
:1003300026EC2AF0B80E3FEC2AF0700E58EC2AF0AA
:10034000100E58EC2AF0100E58EC2AF0100E58EC53
:100350002AF0000E58EC2AF031EC45F0000E58EC73
:100360002AF071EC44F0000E58EC2AF051EC44F005
:10037000000E58EC2AF071EC44F0000E58EC2AF014
:10038000B1EC44F0000E58EC2AF071EC45F0000E90
:1003900058EC2AF071EC44F0000E58EC2AF031ECE5
:1003A00045F061EC47F041EC45F01DEC2AF0400EC1
:1003B00026EC2AF0B80E3FEC2AF051EC45F0000E86
:1003C00058EC2AF031EC44F0000E58EC2AF051ECD5
:1003D00045F0000E58EC2AF061EC45F0000E58ECA8
:1003E0002AF041EC45F0000E58EC2AF0082A210EC4
:1003F000085CD8B401EF02F0100E58EC2AF0F6EFCA
:1004000001F0086A700E58EC2AF01AEC2AF0400E3F
:1004100026EC2AF0BA0E3FEC2AF01DA82CEF02F0D1
:1004200061EC47F061EC47F061EC47F061EC47F0BC
:10043000000E58EC2AF061EC47F0000E58EC2AF060
:1004400061EC47F0000E58EC2AF061EC47F0000E2A
:1004500058EC2AF056EF02F01BA478EF02F0FF0EE2
:1004600058EC2AF091EC46F0FF0E58EC2AF0A1EC83
:1004700046F0FF0E58EC2AF0FF0E58EC2AF0FF0E63
:1004800058EC2AF0E1EC46F0FF0E58EC2AF0E1ECD3
:1004900045F0FF0E58EC2AF081EC46F0FF0E58ECC8
:1004A0002AF0E1EC46F0FF0E58EC2AF0082A1A0E6A
:1004B000085CD8B461EF02F0000E58EC2AF056EF59
:1004C00002F0086A1DEC2AF0400E26EC2AF0BA0E63
:1004D0003FEC2AF0082A070E085CD8B475EF02F04A
:1004E000000E58EC2AF06AEF02F0086AFFEF02F003
:1004F000FF0E58EC2AF0E1EC46F0FF0E58EC2AF023
:10050000E1EC45F0FF0E58EC2AF081EC46F0FF0ECE
:1005100058EC2AF0E1EC46F0FF0E58EC2AF0000E01
:1005200058EC2AF0000E58EC2AF01BA2C8EF02F09B
:10053000FF0E58EC2AF0A1EC46F0FF0E58EC2AF022
:10054000D1EC46F0FF0E58EC2AF041EC46F0FF0EDD
:1005500058EC2AF021EC46F0FF0E58EC2AF091EC12
:1005600046F0FF0E58EC2AF0C1EC45F0FF0E58ECB7
:100570002AF01DEC2AF0400E26EC2AF0BA0E3FECD1
:100580002AF071EC46F0FF0E58EC2AF0FFEF02F073
:10059000FF0E58EC2AF0E1EC45F0FF0E58EC2AF083
:1005A000A1EC46F0FF0E58EC2AF0B1EC46F0FF0E3D
:1005B00058EC2AF041EC47F0FF0E58EC2AF0082ADC
:1005C0000D0E085CD8B4EAEF02F0000E58EC2AF0E9
:1005D000DFEF02F0086A1DEC2AF0400E26EC2AF04C
:1005E000BA0E3FEC2AF0082A070E085CD8B4FEEFDA
:1005F00002F0000E58EC2AF0F3EF02F0086A1DEC4E
:100600002AF0480E26EC2AF0BA0E3FEC2AF01DB86C
:1006100021EF03F01BA621EF03F0FF0E58EC2AF0A8
:10062000B1EC46F0FF0E58EC2AF0D1EC46F0FF0E8C
:1006300058EC2AF0A1EC46F0FF0E58EC2AF02DEF12
:1006400003F0082A140E085CD8B42CEF03F0000E57
:1006500058EC2AF021EF03F0086A1DEC2AF05D0E39
:1006600026EC2AF0BA0E3FEC2AF01DB854EF03F046
:100670001BB054EF03F0FF0E58EC2AF001EC46F0EB
:10068000FF0E58EC2AF081EC46F0FF0E58EC2AF0F1
:10069000B1EC46F0FF0E58EC2AF031EC46F0FF0EBC
:1006A00058EC2AF060EF03F0082A1A0E085CD8B460
:1006B0005FEF03F0000E58EC2AF054EF03F0086AE5
:1006C0001AEC2AF0400E26EC2AF0B90E3FEC2AF084
:1006D0001DB8DFEF04F01CB679EF03F01CB8A7EFEC
:1006E00003F01CBAD5EF03F01CBC05EF04F0DFEFFC
:1006F00004F0FF0E58EC2AF0F1EC45F0FF0E58EC38
:100700002AF0F1EC46F0FF0E58EC2AF0E1EC46F04E
:10071000FF0E58EC2AF0FF0E58EC2AF0FF0EE1EC29
:1007200045F0FF0E58EC2AF0F1EC45F0FF0E58ECC6
:100730002AF0082A110E085CD8B4A4EF03F0000ECA
:1007400058EC2AF099EF03F0086AEBEF04F0FF0E83
:1007500058EC2AF0F1EC45F0FF0E58EC2AF0F1ECE1
:1007600046F0FF0E58EC2AF0E1EC46F0FF0E58EC94
:100770002AF0FF0E58EC2AF0FF0E71EC46F0FF0E47
:1007800058EC2AF0F1EC45F0FF0E58EC2AF0082A5C
:10079000110E085CD8B4D2EF03F0000E58EC2AF02A
:1007A000C7EF03F0086AEBEF04F0FF0E58EC2AF0F5
:1007B00041EC46F0FF0E58EC2AF001EC46F0FF0E3B
:1007C00058EC2AF0E1EC45F0FF0E58EC2AF051EC21
:1007D00042F0FF0E58EC2AF001EC42F0FF0E58EC0C
:1007E0002AF081EC42F0FF0E58EC2AF021EC42F0A6
:1007F000FF0E58EC2AF061EC42F0FF0E58EC2AF0A4
:10080000000E58EC2AF0EBEF04F0FF0E58EC2AF043
:10081000B1EC46F0FF0E58EC2AF0E1EC45F0FF0E8B
:1008200058EC2AF081EC46F0FF0E58EC2AF0000E4E
:1008300058EC2AF02B50526E529E010E525CD8B4E6
:100840003FEF04F0490E525CD8B467EF04F0030E9A
:10085000525CD8B48FEF04F0430E525CD8B4B7EFBB
:1008600004F0082A1E0E085CD8B43CEF04F0000E19
:1008700058EC2AF031EF04F0086AEBEF04F0000EB8
:1008800058EC2AF0FF0E58EC2AF0E1EC45F0FF0E90
:1008900058EC2AF0F1EC45F0FF0E58EC2AF061EC30
:1008A00047F0000E58EC2AF061EC47F0000E58ECCF
:1008B0002AF0000E58EC2AF0000E58EC2AF0000E38
:1008C00058EC2AF0000E58EC2AF0EBEF04F0000E82
:1008D00058EC2AF0FF0E58EC2AF081EC46F0FF0E9F
:1008E00058EC2AF0F1EC45F0FF0E58EC2AF061ECE0
:1008F00047F0000E58EC2AF061EC47F0000E58EC7F
:100900002AF0000E58EC2AF0000E58EC2AF0000EE7
:1009100058EC2AF0000E58EC2AF0EBEF04F0000E31
:1009200058EC2AF0FF0E58EC2AF0F1EC45F0FF0EDF
:1009300058EC2AF0C1EC45F0FF0E58EC2AF0F1EC2F
:1009400046F0FF0E58EC2AF061EC47F0000E58EC30
:100950002AF0000E58EC2AF0000E58EC2AF0000E97
:1009600058EC2AF0000E58EC2AF0EBEF04F0000EE1
:1009700058EC2AF0FF0E58EC2AF0F1EC45F0FF0E8F
:1009800058EC2AF0E1EC45F0FF0E58EC2AF0E1ECCF
:1009900045F0FF0E58EC2AF061EC47F0000E58ECE1
:1009A0002AF0000E58EC2AF0000E58EC2AF0000E47
:1009B00058EC2AF0000E58EC2AF0EBEF04F0082A6D
:1009C000320E085CD8B4EAEF04F0000E58EC2AF0BE
:1009D000DFEF04F0086A1AEC2AF0730E26EC2AF016
:1009E000B90E3FEC2AF01DB829EF05F01CA229EF43
:1009F00005F0FF0E58EC2AF0E1EC46F0FF0E58EC43
:100A00002AF041EC46F0FF0E58EC2AF01DEC2AF0DB
:100A1000400E26EC2AF0B90E3FEC2AF071EC46F0BD
:100A2000FF0E58EC2AF001EC46F0FF0E58EC2AF0CD
:100A300091EC46F0FF0E58EC2AF0E1EC45F0FF0E89
:100A400058EC2AF001EC46F0FF0E58EC2AF049EF82
:100A500005F0082A0E0E085CD8B434EF05F0000E3D
:100A600058EC2AF029EF05F0086A1DEC2AF0400E38
:100A700026EC2AF0B90E3FEC2AF0082A1F0E085C7B
:100A8000D8B448EF05F0000E58EC2AF03DEF05F021
:100A9000086A1DEC2AF0600E26EC2AF0B90E3FEC35
:100AA0002AF01DB879EF05F01CA079EF05F0FF0ED4
:100AB00058EC2AF031EC46F0FF0E58EC2AF041ECED
:100AC00046F0FF0E58EC2AF0FF0E58EC2AF0FF0E0D
:100AD00058EC2AF011EC46F0FF0E58EC2AF0E1EC4D
:100AE00046F0FF0E58EC2AF0000E58EC2AF085EF85
:100AF00005F0082A1C0E085CD8B484EF05F0000E3F
:100B000058EC2AF079EF05F0086A1AEC2AF0400E4A
:100B100026EC2AF0BB0E3FEC2AF04CB095EF05F026
:100B20001D504E6E4F6AAAEF05F01D504E5CD8A4C2
:100B30003F9A000E4F5CD8A4A0EF05F01D504E6EFA
:100B40003FBAAAEF05F0000E4E5CD8B4AAEF05F04C
:100B500027EC39F0000E4E5CD8A4B3EF05F0A5ECFD
:100B600039F0FDEF05F0400E4E5CD8A4BCEF05F067
:100B7000C5EC39F0FDEF05F0200E4E5CD8A4C5EFB2
:100B800005F0E6EC39F0FDEF05F0100E4E5CD8A450
:100B9000CEEF05F007EC3AF0FDEF05F0080E4E5CE5
:100BA000D8A4D7EF05F03FEC3AF0FDEF05F0020EC8
:100BB0004E5CD8A4E0EF05F08DEC3AF0FDEF05F0C7
:100BC000010E4E5CD8A4E9EF05F0DBEC3AF0FDEF46
:100BD00005F0FF0E58EC2AF05BEC3BF04E5058EC61
:100BE00038F0FF0E58EC2AF0FF0E58EC2AF0BAEC61
:100BF00038F061EC47F061EC47F01AEC2AF0400E57
:100C000026EC2AF0BD0E3FEC2AF0000E58EC2AF03C
:100C100081EC44F0000E58EC2AF041EC45F0000E57
:100C200058EC2AF0280E58EC2AF0280E58EC2AF03E
:100C3000280E58EC2AF0280E58EC2AF0280E58EC12
:100C40002AF0000E58EC2AF01AEC2AF0530E26EC8B
:100C50002AF0BD0E3FEC2AF05E0E295CD8A450EFBE
:100C600006F0000E58EC2AF061EC47F0000E58EC4C
:100C70002AF061EC47F0000E58EC2AF0000E58EC18
:100C80002AF0000E58EC2AF081EC41F0000E58ECEE
:100C90002AF071EC41F0000E58EC2AF075EF08F0E4
:100CA0005D0E295CD8A474EF06F0000E58EC2AF013
:100CB00061EC47F0000E58EC2AF061EC47F0000EB2
:100CC00058EC2AF0000E58EC2AF0000E58EC2AF0EE
:100CD00081EC41F0000E58EC2AF071EC41F0000E6E
:100CE00058EC2AF075EF08F0440E295CD8A498EF70
:100CF00006F0000E58EC2AF061EC47F0000E58ECBC
:100D00002AF091EC41F0000E58EC2AF091EC41F001
:100D1000000E58EC2AF0400E58EC2AF0000E58EC69
:100D20002AF061EC41F0000E58EC2AF075EF08F063
:100D3000450E295CD8A4BCEF06F0000E58EC2AF052
:100D400061EC47F0000E58EC2AF091EC41F0000EF7
:100D500058EC2AF091EC41F0000E58EC2AF0400ECD
:100D600058EC2AF0000E58EC2AF061EC41F0000E2D
:100D700058EC2AF075EF08F03E0E295CD8A4E0EF9D
:100D800006F0000E58EC2AF061EC47F0000E58EC2B
:100D90002AF061EC47F0000E58EC2AF0000E58ECF7
:100DA0002AF0000E58EC2AF091EC41F0000E58ECBD
:100DB0002AF0D1EC41F0000E58EC2AF075EF08F063
:100DC0003F0E295CD8A404EF07F0000E58EC2AF07F
:100DD00061EC47F0000E58EC2AF061EC47F0000E91
:100DE00058EC2AF0000E58EC2AF0000E58EC2AF0CD
:100DF00091EC41F0000E58EC2AF0D1EC41F0000EDD
:100E000058EC2AF075EF08F0220E295CD8A428EFE0
:100E100007F0000E58EC2AF061EC47F0FF0E58EC9A
:100E20002AF071EC42F0FF0E58EC2AF071EC42F01F
:100E3000FF0E58EC2AF0BF0E58EC2AF0FF0E58ECCB
:100E40002AF011EC42F0FF0E58EC2AF075EF08F092
:100E5000230E295CD8A44CEF07F0000E58EC2AF0C2
:100E600061EC47F0FF0E58EC2AF071EC42F0FF0EF7
:100E700058EC2AF071EC42F0FF0E58EC2AF0BF0E4D
:100E800058EC2AF0FF0E58EC2AF011EC42F0FF0E5D
:100E900058EC2AF075EF08F01F0E295CD8A470EF0B
:100EA00007F0000E58EC2AF061EC47F0000E58EC09
:100EB0002AF061EC47F0000E58EC2AF0000E58ECD6
:100EC0002AF0FF0E58EC2AF081EC42F0FF0E58ECAD
:100ED0002AF051EC42F0FF0E58EC2AF075EF08F0C2
:100EE000200E295CD8A494EF07F0000E58EC2AF0ED
:100EF00061EC47F0000E58EC2AF061EC47F0000E70
:100F000058EC2AF0000E58EC2AF0FF0E58EC2AF0AC
:100F100081EC42F0FF0E58EC2AF051EC42F0FF0E4B
:100F200058EC2AF075EF08F0110E295CD8A4B8EF40
:100F300007F0FF0E58EC2AF001EC42F0FF0E58ECDF
:100F40002AF061EC42F0FF0E58EC2AF051EC42F02E
:100F5000FF0E58EC2AF0BF0E58EC2AF0FF0E58ECAA
:100F60002AF031EC42F0FF0E58EC2AF075EF08F051
:100F7000120E295CD8A4DCEF07F0FF0E58EC2AF023
:100F800001EC42F0FF0E58EC2AF061EC42F0FF0E4B
:100F900058EC2AF051EC42F0FF0E58EC2AF0BF0E4C
:100FA00058EC2AF0FF0E58EC2AF031EC42F0FF0E1C
:100FB00058EC2AF075EF08F0100E295CD8A400EF69
:100FC00008F0000E58EC2AF061EC47F0000E58ECE7
:100FD0002AF0000E58EC2AF0FF0E58EC2AF001EC33
:100FE00042F0FF0E58EC2AF081EC42F0FF0E58EC74
:100FF0002AF011EC42F0FF0E58EC2AF075EF08F0E1
:101000000F0E295CD8A424EF08F0000E58EC2AF04B
:1010100061EC47F0000E58EC2AF0000E58EC2AF074
:10102000FF0E58EC2AF001EC42F0FF0E58EC2AF0CB
:1010300081EC42F0FF0E58EC2AF011EC42F0FF0E6A
:1010400058EC2AF075EF08F0000E58EC2AF0100E5C
:1010500058EC2AF0100E58EC2AF0100E58EC2AF03A
:10106000100E58EC2AF0100E58EC2AF0000E58EC36
:101070002AF0100E58EC2AF0100E58EC2AF0100E40
:1010800058EC2AF0100E58EC2AF0100E58EC2AF00A
:10109000000E58EC2AF0100E58EC2AF0100E58EC06
:1010A0002AF0100E58EC2AF0100E58EC2AF0100E10
:1010B00058EC2AF0000E58EC2AF0400E58EC2AF0BA
:1010C000000E58EC2AF0100E58EC2AF0100E58ECD6
:1010D0002AF0100E58EC2AF0100E58EC2AF0100EE0
:1010E00058EC2AF0000E58EC2AF0000E58EC2AF0CA
:1010F000C1EC44F0000E58EC2AF0A1EC44F0000ED4
:1011000058EC2AF0B1EC45F0000E58EC2AF01AEC3D
:101110002AF0400E26EC2AF0BC0E3FEC2AF0000E1E
:1011200058EC2AF0B1EC44F0000E58EC2AF0F1EC47
:1011300044F0000E58EC2AF0280E58EC2AF0280E45
:1011400058EC2AF0280E58EC2AF0280E58EC2AF019
:10115000280E58EC2AF0000E58EC2AF01AEC2AF06F
:10116000530E26EC2AF0BC0E3FEC2AF01550380B3B
:10117000406E000E405CD8A4E6EF08F0000E58EC7C
:101180002AF031EC45F0000E58EC2AF091EC45F0D5
:10119000000E58EC2AF011EC45F0000E58EC2AF045
:1011A00051EC41F0000E58EC2AF061EC47F0000ED3
:1011B00058EC2AF061EC47F0000E58EC2AF061EC94
:1011C00047F0000E58EC2AF031EF0AF0080E405CB0
:1011D000D8A413EF09F0000E58EC2AF031EC45F0DA
:1011E000000E58EC2AF091EC45F0000E58EC2AF075
:1011F00011EC45F0000E58EC2AF061EC41F0000EC5
:1012000058EC2AF061EC47F0000E58EC2AF061EC43
:1012100047F0000E58EC2AF061EC47F0000E58EC55
:101220002AF031EF0AF0100E405CD8A440EF09F02C
:10123000000E58EC2AF031EC45F0000E58EC2AF084
:1012400091EC45F0000E58EC2AF011EC45F0000E40
:1012500058EC2AF071EC41F0000E58EC2AF061ECE9
:1012600047F0000E58EC2AF061EC47F0000E58EC05
:101270002AF061EC47F0000E58EC2AF031EF0AF04A
:10128000180E405CD8A484EF09F0000E58EC2AF048
:1012900061EC45F0000E58EC2AF041EC45F0000EF0
:1012A00058EC2AF041EC44F0000E58EC2AF061ECC6
:1012B00047F083A270EF09F0FF0E58EC2AF0C1EC62
:1012C00045F0FF0E58EC2AF0E1EC45F0FF0E58EC2B
:1012D0002AF0F1EC46F0FF0E58EC2AF031EF0AF05C
:1012E000000E58EC2AF041EC45F0000E58EC2AF0C4
:1012F00011EC45F0000E58EC2AF061EC44F0000EC1
:1013000058EC2AF031EF0AF0200E405CD8A4B1EF7F
:1013100009F0000E58EC2AF031EC45F0000E58ECC4
:101320002AF091EC45F0000E58EC2AF011EC45F053
:10133000000E58EC2AF091EC41F0000E58EC2AF027
:1013400061EC47F0000E58EC2AF061EC47F0000E1B
:1013500058EC2AF061EC47F0000E58EC2AF031EF1F
:101360000AF0280E405CD8A4DEEF09F0000E58EC1D
:101370002AF031EC45F0000E58EC2AF091EC45F0E3
:10138000000E58EC2AF011EC45F0000E58EC2AF053
:10139000A1EC41F0000E58EC2AF061EC47F0000E91
:1013A00058EC2AF061EC47F0000E58EC2AF061ECA2
:1013B00047F0000E58EC2AF031EF0AF0300E405C96
:1013C000D8A40BEF0AF0000E58EC2AF031EC45F0EF
:1013D000000E58EC2AF091EC45F0000E58EC2AF083
:1013E00011EC45F0000E58EC2AF0B1EC41F0000E83
:1013F00058EC2AF061EC47F0000E58EC2AF061EC52
:1014000047F0000E58EC2AF061EC47F0000E58EC63
:101410002AF031EF0AF0000E58EC2AF031EC45F0DA
:10142000000E58EC2AF091EC45F0000E58EC2AF032
:1014300011EC45F0000E58EC2AF0C1EC41F0000E22
:1014400058EC2AF061EC47F0000E58EC2AF061EC01
:1014500047F0000E58EC2AF061EC47F0000E58EC13
:101460002AF01DA850921DB84CEF0AF0020E1F5C26
:10147000D8B458EF0AF0030E1F5CD8B458EF0AF046
:10148000010E1F5CD8B458EF0AF0210E1F5CD8B4CF
:1014900058EF0AF052EF0AF050B252EF0AF05FEC48
:1014A0002BF05082206A216A226A236A266A276A00
:1014B000205076EC38F01AEC2AF0400E26EC2AF098
:1014C000BE0E3FEC2AF0080E58EC2AF0F80E58EC4D
:1014D0002AF0080E58EC2AF0E00E58EC2AF0200E04
:1014E00058EC2AF0000E58EC2AF0000E58EC2AF0C6
:1014F000059C92EC38F0215076EC38F01AEC2AF08A
:101500005A0E26EC2AF0BE0E3FEC2AF0F80E58ECEC
:101510002AF0000E58EC2AF0E00E58EC2AF0200ECB
:1015200058EC2AF0E00E58EC2AF0000E58EC2AF0A5
:10153000000E58EC2AF0059C92EC38F0225076EC24
:1015400038F01AEC2AF0400E26EC2AF0BF0E3FECE1
:101550002AF0059C92EC38F081EC47F0235076ECB1
:1015600038F01AEC2AF04E0E26EC2AF0BF0E3FECB3
:101570002AF0059C92EC38F0265076EC38F01AEC04
:101580002AF05C0E26EC2AF0BF0E3FEC2AF0059CF8
:1015900092EC38F081EC47F0275076EC38F01AECFA
:1015A0002AF06A0E26EC2AF0BF0E3FEC2AF0059CCA
:1015B00092EC38F01DEC2AF0460E26EC2AF0BC0E18
:1015C0003FEC2AF0700E58EC2AF0100E58EC2AF07E
:1015D000100E58EC2AF0100E58EC2AF0000E58ECC1
:1015E0002AF091EC44F0000E58EC2AF011EC45F092
:1015F000000E58EC2AF001EC45F0000E58EC2AF0F1
:10160000082A220E085CD8B40BEF0BF0100E58EC31
:101610002AF000EF0BF0086A700E58EC2AF01DEC6F
:101620002AF0460E26EC2AF0BD0E3FEC2AF0000E02
:1016300058EC2AF051EC41F0000E58EC2AF0280E3C
:1016400058EC2AF0280E58EC2AF0280E58EC2AF014
:10165000280E58EC2AF0280E58EC2AF0000E58EC10
:101660002AF013500F0B406EEAEC2DF01DEC2AF01F
:10167000460E26EC2AF0BE0E3FEC2AF0000E58EC87
:101680002AF061EC41F0000E58EC2AF0280E58ECDC
:101690002AF0280E58EC2AF0280E58EC2AF0280ED2
:1016A00058EC2AF0280E58EC2AF0000E58EC2AF0DC
:1016B0001450F00B406E4042404240424042EAEC3F
:1016C0002DF01DEC2AF0460E26EC2AF0BF0E3FEC62
:1016D0002AF0000E58EC2AF071EC41F0000E58ECA4
:1016E0002AF0280E58EC2AF0280E58EC2AF0280E82
:1016F00058EC2AF0280E58EC2AF0280E58EC2AF064
:10170000000E58EC2AF014500F0B406EEAEC2DF04E
:101710001BEF01F04F6A1AEC2AF0410E26EC2AF07A
:10172000B80E3FEC2AF0700E58EC2AF0100E58EC70
:101730002AF0100E58EC2AF0100E58EC2AF0000E89
:1017400058EC2AF051EC44F0000E58EC2AF041EC31
:1017500045F0000E58EC2AF0D1EC41F0000E58ECA8
:101760002AF091EC41F0000E58EC2AF061EC41F0C7
:10177000000E58EC2AF0B1EC41F0000E58EC2AF0C3
:1017800061EC47F031EC45F0000E58EC2AF071ECBA
:1017900044F0000E58EC2AF091EC44F01DEC2AF0D5
:1017A000400E26EC2AF0B80E3FEC2AF0000E58EC62
:1017B0002AF0B1EC44F0000E58EC2AF041EC45F070
:1017C000000E58EC2AF051EC45F0000E58EC2AF0CF
:1017D00071EC44F0000E58EC2AF031EC45F0000EAC
:1017E00058EC2AF0082A200E085CD8B4FDEF0BF064
:1017F000100E58EC2AF0F2EF0BF0086A700E58EC5D
:101800002AF01AEC2AF0410E26EC2AF0B90E3FEC31
:101810002AF0FF0E58EC2AF0C1EC45F0FF0E58EC10
:101820002AF0F1EC45F0FF0E58EC2AF0F1EC45F00F
:10183000FF0E58EC2AF0D1EC46F0FF0E58EC2AF0DF
:1018400001EC46F0FF0E58EC2AF0E1EC46F0FF0EFA
:1018500058EC2AF0E1EC46F0FF0E58EC2AF01DECB3
:101860002AF0410E26EC2AF0B90E3FEC2AF0FF0ECA
:1018700058EC2AF0F1EC45F0FF0E58EC2AF0C1ECE0
:1018800045F0FF0E58EC2AF0F1EC46F0FF0E58EC54
:101890002AF0C1EC45F0FF0E58EC2AF080B062EF60
:1018A0000CF03EB063EF0CF0060E425CD8B45CEF77
:1018B0000CF0422A5DEF0CF0426A42EC2BF03E80C5
:1018C00063EF0CF03E9084B678EF0CF03EBC79EFFD
:1018D0000CF0000E425CD8B471EF0CF0420673EFCE
:1018E0000CF0060E426E42EC2BF03E8C79EF0CF0C1
:1018F0003E9C1AEC2AF0410E26EC2AF0BA0E3FEC80
:101900002AF0000E425CD8B4A6EF0CF0010E425C47
:10191000D8B46CEF0DF0020E425CD8B432EF0EF08A
:10192000030E425CD8B4F8EF0EF0040E425CD8B45B
:10193000BEEF0FF0050E425CD8B484EF10F0060E37
:10194000425CD8B44AEF11F0A8EF11F051EC41F02D
:10195000000E58EC2AF051EC41F0000E58EC2AF041
:10196000A1EC44F0000E58EC2AF01DEC2AF0410ED8
:1019700026EC2AF0BA0E3FEC2AF01150D0EC38F0E9
:101980001AEC2AF0410E26EC2AF0BB0E3FEC2AF0AE
:1019900051EC41F0000E58EC2AF061EC41F0000EE1
:1019A00058EC2AF0A1EC44F0000E58EC2AF01DECA3
:1019B0002AF0410E26EC2AF0BB0E3FEC2AF0125022
:1019C000D0EC38F01AEC2AF0410E26EC2AF0BC0ECE
:1019D0003FEC2AF051EC41F0000E58EC2AF071EC8B
:1019E00041F0000E58EC2AF0A1EC44F0000E58EC47
:1019F0002AF01DEC2AF0410E26EC2AF0BC0E3FEC3A
:101A00002AF01350D0EC38F01AEC2AF0410E26ECF4
:101A10002AF0BD0E3FEC2AF051EC41F0000E58ECDC
:101A20002AF081EC41F0000E58EC2AF0A1EC44F0D1
:101A3000000E58EC2AF01DEC2AF0410E26EC2AF09C
:101A4000BD0E3FEC2AF01450D0EC38F01AEC2AF01E
:101A5000410E26EC2AF0BE0E3FEC2AF051EC41F08C
:101A6000000E58EC2AF091EC41F0000E58EC2AF0F0
:101A7000A1EC44F0000E58EC2AF01DEC2AF0410EC7
:101A800026EC2AF0BE0E3FEC2AF01550D0EC38F0D0
:101A90001AEC2AF0410E26EC2AF0BF0E3FEC2AF099
:101AA00051EC41F0000E58EC2AF0A1EC41F0000E90
:101AB00058EC2AF0A1EC44F0000E58EC2AF01DEC92
:101AC0002AF0410E26EC2AF0BF0E3FEC2AF0165009
:101AD000D0EC38F0A8EF11F051EC41F0000E58ECCA
:101AE0002AF0B1EC41F0000E58EC2AF0A1EC44F0E1
:101AF000000E58EC2AF01DEC2AF0410E26EC2AF0DC
:101B0000BA0E3FEC2AF01750D0EC38F01AEC2AF05D
:101B1000410E26EC2AF0BB0E3FEC2AF051EC41F0CE
:101B2000000E58EC2AF0C1EC41F0000E58EC2AF0FF
:101B3000A1EC44F0000E58EC2AF01DEC2AF0410E06
:101B400026EC2AF0BB0E3FEC2AF01850D0EC38F00F
:101B50001AEC2AF0410E26EC2AF0BC0E3FEC2AF0DB
:101B600051EC41F0000E58EC2AF0D1EC41F0000E9F
:101B700058EC2AF0A1EC44F0000E58EC2AF01DECD1
:101B80002AF0410E26EC2AF0BC0E3FEC2AF0195048
:101B9000D0EC38F01AEC2AF0410E26EC2AF0BD0EFB
:101BA0003FEC2AF051EC41F0000E58EC2AF0E1EC49
:101BB00041F0000E58EC2AF0A1EC44F0000E58EC75
:101BC0002AF01DEC2AF0410E26EC2AF0BD0E3FEC67
:101BD0002AF01A50D0EC38F01AEC2AF0410E26EC1C
:101BE0002AF0BE0E3FEC2AF051EC41F0000E58EC0A
:101BF0002AF031EC44F0000E58EC2AF0A1EC44F04D
:101C0000000E58EC2AF01DEC2AF0410E26EC2AF0CA
:101C1000BE0E3FEC2AF01B50D0EC38F01AEC2AF044
:101C2000410E26EC2AF0BF0E3FEC2AF051EC41F0B9
:101C3000000E58EC2AF041EC44F0000E58EC2AF06B
:101C4000A1EC44F0000E58EC2AF01DEC2AF0410EF5
:101C500026EC2AF0BF0E3FEC2AF01C50D0EC38F0F6
:101C6000A8EF11F051EC41F0000E58EC2AF051ECC5
:101C700044F0000E58EC2AF0A1EC44F0000E58ECB1
:101C80002AF01DEC2AF0410E26EC2AF0BA0E3FECA9
:101C90002AF01D50D0EC38F01AEC2AF0410E26EC58
:101CA0002AF0BB0E3FEC2AF051EC41F0000E58EC4C
:101CB0002AF061EC44F0000E58EC2AF0A1EC44F05C
:101CC000000E58EC2AF01DEC2AF0410E26EC2AF00A
:101CD000BB0E3FEC2AF01E50D0EC38F01AEC2AF084
:101CE000410E26EC2AF0BC0E3FEC2AF051EC41F0FC
:101CF000000E58EC2AF071EC44F0000E58EC2AF07B
:101D0000A1EC44F0000E58EC2AF01DEC2AF0410E34
:101D100026EC2AF0BC0E3FEC2AF01F50D0EC38F035
:101D20001AEC2AF0410E26EC2AF0BD0E3FEC2AF008
:101D300051EC41F0000E58EC2AF081EC44F0000E1A
:101D400058EC2AF0A1EC44F0000E58EC2AF01DECFF
:101D50002AF0410E26EC2AF0BD0E3FEC2AF020506E
:101D6000D0EC38F01AEC2AF0410E26EC2AF0BE0E28
:101D70003FEC2AF061EC41F0000E58EC2AF051ECF7
:101D800041F0000E58EC2AF0A1EC44F0000E58ECA3
:101D90002AF01DEC2AF0410E26EC2AF0BE0E3FEC94
:101DA0002AF02150D0EC38F01AEC2AF0410E26EC43
:101DB0002AF0BF0E3FEC2AF061EC41F0000E58EC27
:101DC0002AF061EC41F0000E58EC2AF0A1EC44F04E
:101DD000000E58EC2AF01DEC2AF0410E26EC2AF0F9
:101DE000BF0E3FEC2AF02250D0EC38F0A8EF11F0F3
:101DF00061EC41F0000E58EC2AF071EC41F0000E5D
:101E000058EC2AF0A1EC44F0000E58EC2AF01DEC3E
:101E10002AF0410E26EC2AF0BA0E3FEC2AF02350AD
:101E2000D0EC38F01AEC2AF0410E26EC2AF0BB0E6A
:101E30003FEC2AF061EC41F0000E58EC2AF081EC06
:101E400041F0000E58EC2AF0A1EC44F0000E58ECE2
:101E50002AF01DEC2AF0410E26EC2AF0BB0E3FECD6
:101E60002AF02450D0EC38F01AEC2AF0410E26EC7F
:101E70002AF0BC0E3FEC2AF061EC41F0000E58EC69
:101E80002AF091EC41F0000E58EC2AF0A1EC44F05D
:101E9000000E58EC2AF01DEC2AF0410E26EC2AF038
:101EA000BC0E3FEC2AF02550D0EC38F01AEC2AF0AA
:101EB000410E26EC2AF0BD0E3FEC2AF061EC41F019
:101EC000000E58EC2AF0A1EC41F0000E58EC2AF07C
:101ED000A1EC44F0000E58EC2AF01DEC2AF0410E63
:101EE00026EC2AF0BD0E3FEC2AF02650D0EC38F05C
:101EF0001AEC2AF0410E26EC2AF0BE0E3FEC2AF036
:101F000061EC41F0000E58EC2AF0B1EC41F0000E0B
:101F100058EC2AF0A1EC44F0000E58EC2AF01DEC2D
:101F20002AF0410E26EC2AF0BE0E3FEC2AF0275094
:101F3000D0EC38F01AEC2AF0410E26EC2AF0BF0E55
:101F40003FEC2AF061EC41F0000E58EC2AF0C1ECB5
:101F500041F0000E58EC2AF0A1EC44F0000E58ECD1
:101F60002AF01DEC2AF0410E26EC2AF0BF0E3FECC1
:101F70002AF02850D0EC38F0A8EF11F061EC41F0D5
:101F8000000E58EC2AF0D1EC41F0000E58EC2AF08B
:101F9000A1EC44F0000E58EC2AF01DEC2AF0410EA2
:101FA00026EC2AF0BA0E3FEC2AF02950D0EC38F09B
:101FB0001AEC2AF0410E26EC2AF0BB0E3FEC2AF078
:101FC00061EC41F0000E58EC2AF0E1EC41F0000E1B
:101FD00058EC2AF0A1EC44F0000E58EC2AF01DEC6D
:101FE0002AF0410E26EC2AF0BB0E3FEC2AF02A50D4
:101FF000D0EC38F01AEC2AF0410E26EC2AF0BC0E98
:102000003FEC2AF061EC41F0000E58EC2AF031EC84
:1020100044F0000E58EC2AF0A1EC44F0000E58EC0D
:102020002AF01DEC2AF0410E26EC2AF0BC0E3FEC03
:102030002AF02B50D0EC38F01AEC2AF0410E26ECA6
:102040002AF0BD0E3FEC2AF061EC41F0000E58EC96
:102050002AF041EC44F0000E58EC2AF0A1EC44F0D8
:10206000000E58EC2AF01DEC2AF0410E26EC2AF066
:10207000BD0E3FEC2AF02C50D0EC38F01AEC2AF0D0
:10208000410E26EC2AF0BE0E3FEC2AF061EC41F046
:10209000000E58EC2AF051EC44F0000E58EC2AF0F7
:1020A000A1EC44F0000E58EC2AF01DEC2AF0410E91
:1020B00026EC2AF0BE0E3FEC2AF02D50D0EC38F082
:1020C0001AEC2AF0410E26EC2AF0BF0E3FEC2AF063
:1020D00061EC41F0000E58EC2AF061EC44F0000E87
:1020E00058EC2AF0A1EC44F0000E58EC2AF01DEC5C
:1020F0002AF0410E26EC2AF0BF0E3FEC2AF02E50BB
:10210000D0EC38F0A8EF11F061EC41F0000E58EC83
:102110002AF071EC44F0000E58EC2AF0A1EC44F0E7
:10212000000E58EC2AF01DEC2AF0410E26EC2AF0A5
:10213000BA0E3FEC2AF02F50D0EC38F01AEC2AF00F
:10214000410E26EC2AF0BB0E3FEC2AF061EC41F088
:10215000000E58EC2AF081EC44F0000E58EC2AF006
:10216000A1EC44F0000E58EC2AF01DEC2AF0410ED0
:1021700026EC2AF0BB0E3FEC2AF03050D0EC38F0C1
:102180001AEC2AF0410E26EC2AF0BC0E3FEC2AF0A5
:1021900071EC41F0000E58EC2AF051EC41F0000EC9
:1021A00058EC2AF0A1EC44F0000E58EC2AF01DEC9B
:1021B0002AF0410E26EC2AF0BC0E3FEC2AF03150FA
:1021C000D0EC38F01AEC2AF0410E26EC2AF0BD0EC5
:1021D0003FEC2AF071EC41F0000E58EC2AF061EC73
:1021E00041F0000E58EC2AF0A1EC44F0000E58EC3F
:1021F0002AF01DEC2AF0410E26EC2AF0BD0E3FEC31
:102200002AF03250D0EC38F01AEC2AF0410E26ECCD
:102210002AF0BE0E3FEC2AF071EC41F0000E58ECB3
:102220002AF071EC41F0000E58EC2AF0A1EC44F0D9
:10223000000E58EC2AF01DEC2AF0410E26EC2AF094
:10224000BE0E3FEC2AF03350D0EC38F01AEC2AF0F6
:10225000410E26EC2AF0BF0E3FEC2AF071EC41F063
:10226000000E58EC2AF081EC41F0000E58EC2AF0F8
:10227000A1EC44F0000E58EC2AF01DEC2AF0410EBF
:1022800026EC2AF0BF0E3FEC2AF03450D0EC38F0A8
:10229000A8EF11F071EC41F0000E58EC2AF091EC2F
:1022A00041F0000E58EC2AF0A1EC44F0000E58EC7E
:1022B0002AF01DEC2AF0410E26EC2AF0BA0E3FEC73
:1022C0002AF03550D0EC38F01AEC2AF0410E26EC0A
:1022D0002AF0BB0E3FEC2AF071EC41F0000E58ECF6
:1022E0002AF0A1EC41F0000E58EC2AF0A1EC44F0E9
:1022F000000E58EC2AF01DEC2AF0410E26EC2AF0D4
:10230000BB0E3FEC2AF03650D0EC38F01AEC2AF035
:10231000410E26EC2AF0BC0E3FEC2AF071EC41F0A5
:10232000000E58EC2AF0B1EC41F0000E58EC2AF007
:10233000A1EC44F0000E58EC2AF01DEC2AF0410EFE
:1023400026EC2AF0BC0E3FEC2AF03750D0EC38F0E7
:10235000DBEC2DF01BEF01F01AEC2AF0410E26EC1D
:102360002AF0B80E3FEC2AF0700E58EC2AF0100E4E
:1023700058EC2AF0100E58EC2AF0100E58EC2AF007
:10238000000E58EC2AF051EC44F0000E58EC2AF004
:1023900041EC45F0000E58EC2AF0D1EC41F0000E73
:1023A00058EC2AF091EC41F0000E58EC2AF061EC68
:1023B00041F0000E58EC2AF0B1EC41F0000E58EC60
:1023C0002AF061EC47F041EC45F0000E58EC2AF0A1
:1023D00071EC44F0000E58EC2AF051EC45F01DEC85
:1023E0002AF0400E26EC2AF0B80E3FEC2AF0000E40
:1023F00058EC2AF051EC45F0000E58EC2AF0B1EC04
:1024000044F0000E58EC2AF0F1EC44F0000E58ECC9
:102410002AF091EC44F0000E58EC2AF0082A260E1F
:10242000085CD8B419EF12F0100E58EC2AF00EEF39
:1024300012F0086A700E58EC2AF0000E435CD8B413
:1024400029EF12F0010E435CD8B44BEF15F01BEFEF
:1024500001F01AEC2AF0460E26EC2AF0B90E3FECF9
:102460002AF041EC45F0000E58EC2AF071EC44F0F3
:10247000000E58EC2AF0D1EC44F0000E58EC2AF093
:1024800071EC44F0000E58EC2AF051EC44F0000ED0
:1024900058EC2AF051EC45F0000E58EC2AF061ECB3
:1024A00047F031EC44F0000E58EC2AF061EC44F0B7
:1024B000000E58EC2AF061EC44F01DEC2AF0400EBE
:1024C00026EC2AF0B90E3FEC2AF0000E58EC2AF068
:1024D00031EC45F0000E58EC2AF071EC44F0000E9F
:1024E00058EC2AF041EC45F0000E58EC2AF041EC93
:1024F00045F0000E58EC2AF080B08EEF12F03EB09E
:102500008FEF12F00A0E465CD8B48AEF12F0462A1A
:102510008BEF12F0466A3E808FEF12F03E9084B649
:10252000A2EF12F03EBCA3EF12F0000E465CD8B44E
:102530009DEF12F046069FEF12F00A0E466E3E8C9B
:10254000A3EF12F03E9C3F941AEC2AF04A0E26ECC0
:102550002AF0BB0E3FEC2AF0000E465CD8B4C5EF63
:1025600012F0000E58EC2AF051EC41F0000E58EC3D
:102570002AF051EC41F0000E58EC2AF0A1EC44F0A6
:10258000000E58EC2AF0D7EF12F0FF0E58EC2AF0AC
:10259000F1EC41F0FF0E58EC2AF0F1EC41F0FF0EA7
:1025A00058EC2AF031EC46F0FF0E58EC2AF01AEC09
:1025B0002AF0670E26EC2AF0BB0E3FEC2AF0010E43
:1025C000465CD8B4F8EF12F0000E58EC2AF051EC4B
:1025D00041F0000E58EC2AF061EC41F0000E58EC8E
:1025E0002AF0A1EC44F0000E58EC2AF00AEF13F0A8
:1025F000FF0E58EC2AF0F1EC41F0FF0E58EC2AF0F7
:1026000001EC42F0FF0E58EC2AF031EC46F0FF0EE0
:1026100058EC2AF01DEC2AF0440E26EC2AF0BB0EF2
:102620003FEC2AF0020E465CD8B42BEF13F0000EFC
:1026300058EC2AF051EC41F0000E58EC2AF071EC05
:1026400041F0000E58EC2AF0A1EC44F0000E58ECDA
:102650002AF03DEF13F0FF0E58EC2AF0F1EC41F0B8
:10266000FF0E58EC2AF011EC42F0FF0E58EC2AF065
:1026700031EC46F0FF0E58EC2AF01DEC2AF0610E0A
:1026800026EC2AF0BB0E3FEC2AF0030E465CD8B4D1
:102690005EEF13F0000E58EC2AF051EC41F0000E02
:1026A00058EC2AF081EC41F0000E58EC2AF0A1EC35
:1026B00044F0000E58EC2AF070EF13F0FF0E58ECC7
:1026C0002AF0F1EC41F0FF0E58EC2AF021EC42F038
:1026D000FF0E58EC2AF031EC46F0FF0E58EC2AF0D1
:1026E0001AEC2AF04A0E26EC2AF0BC0E3FEC2AF037
:1026F000040E465CD8B491EF13F0000E58EC2AF0AB
:1027000051EC41F0000E58EC2AF091EC41F0000E33
:1027100058EC2AF0A1EC44F0000E58EC2AF0A3EF9C
:1027200013F0FF0E58EC2AF0F1EC41F0FF0E58ECDC
:102730002AF031EC42F0FF0E58EC2AF031EC46F072
:10274000FF0E58EC2AF01AEC2AF0670E26EC2AF05D
:10275000BC0E3FEC2AF0050E465CD8B4C4EF13F073
:10276000000E58EC2AF051EC41F0000E58EC2AF023
:10277000A1EC41F0000E58EC2AF0A1EC44F0000E60
:1027800058EC2AF0D6EF13F0FF0E58EC2AF0F1ECDB
:1027900041F0FF0E58EC2AF041EC42F0FF0E58ECED
:1027A0002AF031EC46F0FF0E58EC2AF01DEC2AF02E
:1027B000440E26EC2AF0BC0E3FEC2AF0060E465CD6
:1027C000D8B4F7EF13F0000E58EC2AF051EC41F0BA
:1027D000000E58EC2AF0B1EC41F0000E58EC2AF053
:1027E000A1EC44F0000E58EC2AF009EF14F0FF0EB3
:1027F00058EC2AF0F1EC41F0FF0E58EC2AF051ECC5
:1028000042F0FF0E58EC2AF031EC46F0FF0E58EC87
:102810002AF01DEC2AF0610E26EC2AF0B40E3FECF3
:102820002AF0070E465CD8B42AEF14F0000E58ECDC
:102830002AF051EC41F0000E58EC2AF0C1EC41F0C6
:10284000000E58EC2AF0A1EC44F0000E58EC2AF0EF
:102850003CEF14F0FF0E58EC2AF0F1EC41F0FF0EC3
:1028600058EC2AF061EC42F0FF0E58EC2AF031EC03
:1028700046F0FF0E58EC2AF01AEC2AF04A0E26EC2D
:102880002AF0BD0E3FEC2AF0080E465CD8B45DEF8E
:1028900014F0000E58EC2AF051EC41F0000E58EC08
:1028A0002AF0D1EC41F0000E58EC2AF0A1EC44F0F3
:1028B000000E58EC2AF06FEF14F0FF0E58EC2AF0DF
:1028C000F1EC41F0FF0E58EC2AF071EC42F0FF0EF3
:1028D00058EC2AF031EC46F0FF0E58EC2AF01AECD6
:1028E0002AF0670E26EC2AF0BD0E3FEC2AF0090E06
:1028F000465CD8B490EF14F0000E58EC2AF051EC7E
:1029000041F0000E58EC2AF0E1EC41F0000E58ECDA
:102910002AF0A1EC44F0000E58EC2AF0A2EF14F0DB
:10292000FF0E58EC2AF0F1EC41F0FF0E58EC2AF0C3
:1029300081EC42F0FF0E58EC2AF031EC46F0FF0E2D
:1029400058EC2AF01AEC2AF04A0E26EC2AF0BF0EB8
:102950003FEC2AF00A0E465CD8B4F5EF14F0000EF6
:1029600058EC2AF061EC44F0000E58EC2AF071ECBF
:1029700044F0000E58EC2AF081EC44F0000E58ECC4
:102980002AF031EC44F0000E58EC2AF061EC45F0EE
:10299000000E58EC2AF0D1EC44F0000E58EC2AF06E
:1029A00051EC45F0000E58EC2AF061EC47F0D1EC08
:1029B00044F0000E58EC2AF01DEC2AF0400E26ECF4
:1029C0002AF0BF0E3FEC2AF001EC45F0000E58EC67
:1029D0002AF031EC44F0000E58EC2AF061EC44F09F
:1029E000000E58EC2AF039EF15F0FF0E58EC2AF0E3
:1029F000F1EC45F0FF0E58EC2AF001EC46F0FF0E2A
:102A000058EC2AF011EC46F0FF0E58EC2AF0C1EC1D
:102A100045F0FF0E58EC2AF001EC47F0FF0E58ECA1
:102A20002AF071EC46F0FF0E58EC2AF0F1EC46F07B
:102A3000FF0E58EC2AF071EC47F071EC46F0FF0EF7
:102A400058EC2AF01DEC2AF0400E26EC2AF0BF0EBE
:102A50003FEC2AF0A1EC46F0FF0E58EC2AF0C1EC56
:102A600045F0FF0E58EC2AF0F1EC45F0FF0E58EC63
:102A70002AF0DBEC2DF080B848EF15F03EB849EFB6
:102A800015F0010E436E42EC2BF03E8849EF15F035
:102A90003E981BEF01F01AEC2AF0460E26EC2AF0C5
:102AA000B90E3FEC2AF0000E465CD8B487EF15F063
:102AB000010E465CD8B474EF16F0020E465CD8B432
:102AC000CDEF17F0030E465CD8B4E1EF18F0040E1A
:102AD000465CD8B4C5EF19F0050E465CD8B4D4EF07
:102AE0001AF0060E465CD8B4FBEF1BF0070E465CEE
:102AF000D8B45FEF1DF0080E465CD8B417EF1EF097
:102B0000090E465CD8B4CFEF1EF087EF1FF09EECA5
:102B10003BF03FB28EEF15F0050E496E3FB4DDEF8E
:102B200015F080B0B6EF15F03EB0B7EF15F0010E1E
:102B3000495CD8A4A0EF15F0080E496EB3EF15F06C
:102B4000040E495CD8A4A9EF15F0010E496EB3EF4D
:102B500015F0080E495CD8A4B2EF15F0050E496EC9
:102B6000B3EF15F049063E80B7EF15F03E9084B6FE
:102B7000DCEF15F03EBCDDEF15F0080E495CD8A483
:102B8000C6EF15F0010E496ED9EF15F0010E495C44
:102B9000D8A4CFEF15F0040E496ED9EF15F0050E4D
:102BA000495CD8A4D8EF15F0080E496ED9EF15F09E
:102BB000492A3E8CDDEF15F03E9C1AEC2AF0460EB9
:102BC00026EC2AF0BC0E3FEC2AF0010E495CD8B48A
:102BD00017EF16F0040E495CD8B43AEF16F0080E61
:102BE000495CD8B45BEF16F0FF0E58EC2AF0F1EC1C
:102BF00046F0FF0E58EC2AF0D1EC46F0FF0E58ECF0
:102C00002AF001EC47F0FF0E58EC2AF091EC46F068
:102C1000FF0E58EC2AF0E1EC45F0FF0E58EC2AF0DC
:102C200061EC47F0000E58EC2AF05BEF16F0FF0E57
:102C300058EC2AF011EC46F0FF0E58EC2AF0E1ECCB
:102C400046F0FF0E58EC2AF021EC47F0FF0E58EC4E
:102C50002AF0E1EC45F0FF0E58EC2AF071EC46F05A
:102C6000FF0E58EC2AF061EC46F0FF0E58EC2AF00B
:102C70005BEF16F0FF0E58EC2AF0B1EC46F0FF0EB9
:102C800058EC2AF0F1EC45F0FF0E58EC2AF001EC7C
:102C900047F0FF0E58EC2AF0D1EC46F0FF0E58EC4E
:102CA0002AF061EC47F0000E58EC2AF061EC47F096
:102CB000000E58EC2AF03FB662EF16F03F86115036
:102CC0004A6E4B6E57EC31F01DEC2AF0400E26ECAC
:102CD0002AF0BD0E3FEC2AF04050E8EC38F031EC21
:102CE00039F03F8274EF20F0F7EC3BF03FB27BEF1E
:102CF00016F0070E496E3FA405EC31F01AEC2AF0ED
:102D0000460E26EC2AF0BC0E3FEC2AF0000E495C81
:102D1000D8B4D6EF16F0010E495CD8B4FEEF16F029
:102D2000020E495CD8B426EF17F0030E495CD8B404
:102D300026EF17F0040E495CD8B45AEF17F0050ED1
:102D4000495CD8B45AEF17F0060E495CD8B48EEF40
:102D500017F0080E495CD8B4B4EF17F0FF0E58EC2A
:102D60002AF0E1EC45F0FF0E58EC2AF031EC46F089
:102D7000FF0E58EC2AF0E1EC46F0FF0E58EC2AF07A
:102D800061EC47F0000E58EC2AF061EC47F0000EC1
:102D900058EC2AF061EC47F0000E58EC2AF061EC98
:102DA00047F0000E58EC2AF0B4EF17F0FF0E58EC85
:102DB0002AF0E1EC46F0FF0E58EC2AF021EC47F047
:102DC000FF0E58EC2AF0E1EC45F0FF0E58EC2AF02B
:102DD00071EC46F0FF0E58EC2AF061EC46F0FF0E65
:102DE00058EC2AF061EC47F0000E58EC2AF061EC48
:102DF00047F0000E58EC2AF0B4EF17F0FF0E58EC35
:102E00002AF081EC46F0FF0E58EC2AF001EC47F076
:102E1000FF0E58EC2AF0F1EC46F0FF0E58EC2AF0C9
:102E200001EC46F0FF0E58EC2AF0E1EC46F0FF0E04
:102E300058EC2AF0C1EC45F0FF0E58EC2AF0A1EC5A
:102E400046F0FF0E58EC2AF0B4EF17F0FF0E58ECE6
:102E50002AF041EC46F0FF0E58EC2AF091EC46F0D7
:102E6000FF0E58EC2AF0F1EC46F0FF0E58EC2AF079
:102E7000020E495CD8B444EF17F0F1EC41F0FF0EBC
:102E800058EC2AF049EF17F001EC42F0FF0E58EC35
:102E90002AF061EC47F0000E58EC2AF061EC47F0A4
:102EA000000E58EC2AF061EC47F0000E58EC2AF0C6
:102EB000B4EF17F0FF0E58EC2AF031EC46F0FF0E9D
:102EC00058EC2AF0A1EC46F0FF0E58EC2AF071EC19
:102ED00046F0FF0E58EC2AF0F1EC45F0FF0E58ECEE
:102EE0002AF0040E495CD8B47DEF17F0F1EC41F004
:102EF000FF0E58EC2AF082EF17F001EC42F0FF0EC3
:102F000058EC2AF061EC47F0000E58EC2AF061EC26
:102F100047F0000E58EC2AF0B4EF17F0FF0E58EC13
:102F20002AF0D1EC46F0FF0E58EC2AF081EC46F086
:102F3000FF0E58EC2AF0E1EC45F0FF0E58EC2AF0B9
:102F400061EC46F0FF0E58EC2AF011EC46F0FF0E53
:102F500058EC2AF061EC47F0000E58EC2AF061ECD6
:102F600047F0000E58EC2AF03FB6BBEF17F03F8653
:102F700012504A6E4B6E57EC31F01DEC2AF0400EA9
:102F800026EC2AF0BD0E3FEC2AF04050E8EC38F079
:102F900031EC39F03F8274EF20F050EC3CF03FB25E
:102FA000D4EF17F0070E496E3FA405EC31F01AEC90
:102FB0002AF0460E26EC2AF0BC0E3FEC2AF0000E5A
:102FC000495CD8B44EEF18F0010E495CD8B480EFDC
:102FD00018F0020E495CD8B480EF18F0030E495C7B
:102FE000D8B480EF18F0080E495CD8B4C8EF18F0D8
:102FF000FF0E58EC2AF021EC46F0FF0E58EC2AF0B8
:10300000B1EC46F0FF0E58EC2AF0A1EC46F0FF0EB2
:1030100058EC2AF0F1EC41F0FF0E58EC2AF0E1EC0C
:1030200046F0FF0E58EC2AF001EC46F0FF0E58EC8B
:103030002AF071EC46F0FF0E58EC2AF0040E495CC1
:10304000D8B434EF18F0050E495CD8B43BEF18F053
:10305000060E495CD8B442EF18F0F1EC41F0FF0ED7
:1030600058EC2AF047EF18F021EC42F0FF0E58EC34
:103070002AF047EF18F011EC42F0FF0E58EC2AF05E
:1030800047EF18F001EC42F0FF0E58EC2AF061EC2B
:1030900047F0000E58EC2AF0C8EF18F0FF0E58EC7D
:1030A0002AF0F1EC45F0FF0E58EC2AF001EC46F066
:1030B000FF0E58EC2AF0F1EC46F0FF0E58EC2AF027
:1030C000E1EC45F0FF0E58EC2AF041EC46F0FF0E23
:1030D00058EC2AF061EC47F0000E58EC2AF061EC55
:1030E00047F0000E58EC2AF061EC47F0000E58EC67
:1030F0002AF061EC47F0000E58EC2AF0C8EF18F007
:10310000FF0E58EC2AF001EC46F0FF0E58EC2AF0C6
:1031100081EC46F0FF0E58EC2AF0B1EC46F0FF0EC1
:1031200058EC2AF031EC46F0FF0E58EC2AF0E1ECB6
:1031300045F0FF0E58EC2AF091EC46F0FF0E58ECEB
:103140002AF0F1EC46F0FF0E58EC2AF071EC46F054
:10315000FF0E58EC2AF0010E495CD8B4BCEF18F011
:10316000020E495CD8B4C3EF18F0F1EC41F0FF0E49
:1031700058EC2AF0C8EF18F011EC42F0FF0E58ECB2
:103180002AF0C8EF18F001EC42F0FF0E58EC2AF0DC
:103190003FB6CFEF18F03F8613504A6E4B6E57EC98
:1031A00031F01DEC2AF0400E26EC2AF0BD0E3FEC6B
:1031B0002AF04050E8EC38F031EC39F03F8274EFFF
:1031C00020F0A9EC3CF03FB2E8EF18F0070E496E92
:1031D0003FA405EC31F01AEC2AF0460E26EC2AF05A
:1031E000BC0E3FEC2AF0000E495CD8B45DEF19F03C
:1031F000010E495CD8B45DEF19F0020E495CD8B4F9
:103200005DEF19F0030E495CD8B45DEF19F0080EBC
:10321000495CD8B4ACEF19F0FF0E58EC2AF021EC61
:1032200046F0FF0E58EC2AF0B1EC46F0FF0E58ECD9
:103230002AF0A1EC46F0FF0E58EC2AF011EC42F017
:10324000FF0E58EC2AF0E1EC46F0FF0E58EC2AF0A5
:1032500001EC46F0FF0E58EC2AF071EC46F0FF0E40
:1032600058EC2AF0040E495CD8B448EF19F0050E6A
:10327000495CD8B44FEF19F0060E495CD8B456EF4C
:1032800019F0F1EC41F0FF0E58EC2AF0ACEF19F018
:1032900021EC42F0FF0E58EC2AF0ACEF19F011ECE3
:1032A00042F0FF0E58EC2AF0ACEF19F001EC42F0BE
:1032B000FF0E58EC2AF0ACEF19F0FF0E58EC2AF094
:1032C00021EC46F0FF0E58EC2AF0B1EC46F0FF0E70
:1032D00058EC2AF0A1EC46F0FF0E58EC2AF001EC75
:1032E00042F0FF0E58EC2AF0E1EC46F0FF0E58ECED
:1032F0002AF001EC46F0FF0E58EC2AF071EC46F093
:10330000FF0E58EC2AF0000E495CD8B499EF19F082
:10331000010E495CD8B4A0EF19F0020E495CD8B494
:10332000A7EF19F0F1EC41F0FF0E58EC2AF0ACEFEA
:1033300019F021EC42F0FF0E58EC2AF0ACEF19F036
:1033400011EC42F0FF0E58EC2AF0ACEF19F001EC52
:1033500042F0FF0E58EC2AF03FB6B3EF19F03F866B
:1033600014504A6E4B6E57EC31F01DEC2AF0400EB3
:1033700026EC2AF0BD0E3FEC2AF04050E8EC38F085
:1033800031EC39F03F8274EF20F002EC3DF03FB2B7
:10339000CCEF19F0070E496E3FA405EC31F01AECA2
:1033A0002AF0460E26EC2AF0BC0E3FEC2AF0000E66
:1033B000495CD8B401EF1AF0010E495CD8B424EF8F
:1033C0001AF0020E495CD8B447EF1AF0030E495CBC
:1033D000D8B447EF1AF0040E495CD8B447EF1AF09E
:1033E000050E495CD8B482EF1AF0060E495CD8B4D9
:1033F00082EF1AF0080E495CD8B4BBEF1AF082EFE6
:103400001AF0FF0E58EC2AF0D1EC46F0FF0E58EC03
:103410002AF001EC47F0FF0E58EC2AF091EC46F050
:10342000FF0E58EC2AF061EC47F0000E58EC2AF041
:1034300061EC47F0000E58EC2AF061EC47F0000E0A
:1034400058EC2AF0BBEF1AF0FF0E58EC2AF0D1EC42
:1034500046F0FF0E58EC2AF031EC47F0FF0E58EC26
:103460002AF0F1EC45F0FF0E58EC2AF061EC47F041
:10347000000E58EC2AF061EC47F0000E58EC2AF0F0
:1034800061EC47F0000E58EC2AF0BBEF1AF0FF0E8B
:1034900058EC2AF0D1EC46F0FF0E58EC2AF031EC53
:1034A00047F0FF0E58EC2AF0E1EC46F0FF0E58EC26
:1034B0002AF001EC46F0FF0E58EC2AF071EC46F0D1
:1034C000FF0E58EC2AF0020E495CD8B474EF1AF0E3
:1034D000030E495CD8B47BEF1AF0F1EC41F0FF0E1B
:1034E00058EC2AF0BBEF1AF011EC42F0FF0E58EC4A
:1034F0002AF0BBEF1AF001EC42F0FF0E58EC2AF074
:10350000BBEF1AF0FF0E58EC2AF0F1EC46F0FF0E7C
:1035100058EC2AF031EC47F0FF0E58EC2AF0E1ECC1
:1035200046F0FF0E58EC2AF001EC46F0FF0E58EC86
:103530002AF071EC46F0FF0E58EC2AF0050E495CBB
:10354000D8B4AFEF1AF0060E495CD8B4B6EF1AF053
:10355000F1EC41F0FF0E58EC2AF0BBEF1AF011EC41
:1035600042F0FF0E58EC2AF0BBEF1AF001EC42F0EB
:10357000FF0E58EC2AF03FB6C2EF1AF03F86155006
:103580004A6E4B6E57EC31F01DEC2AF0400E26ECE3
:103590002AF0BD0E3FEC2AF04050E8EC38F031EC58
:1035A00039F03F8274EF20F05BEC3DF03FB2DBEF8F
:1035B0001AF0070E496E3FA405EC31F01AEC2AF020
:1035C000460E26EC2AF0BC0E3FEC2AF0080E495CB1
:1035D000D8B4E2EF1BF0FF0E58EC2AF0E1EC46F015
:1035E000FF0E58EC2AF0A1EC46F0FF0E58EC2AF042
:1035F000000E495CD8B436EF1BF0010E495CD8B41C
:1036000051EF1BF0020E495CD8B46CEF1BF0030EB7
:10361000495CD8B46CEF1BF0040E495CD8B493EF4E
:103620001BF0050E495CD8B4AEEF1BF0060E495CEA
:10363000D8B4C9EF1BF071EC46F0FF0E58EC2AF03D
:10364000D1EC46F0FF0E58EC2AF0B1EC46F0FF0E3C
:1036500058EC2AF0A1EC46F0FF0E58EC2AF071EC81
:1036600046F0FF0E58EC2AF0E2EF1BF081EC46F03A
:10367000FF0E58EC2AF0E1EC46F0FF0E58EC2AF071
:1036800061EC47F0000E58EC2AF061EC47F0000EB8
:1036900058EC2AF061EC47F0000E58EC2AF0E2EF0B
:1036A0001BF0E1EC46F0FF0E58EC2AF011EC46F06E
:1036B000FF0E58EC2AF061EC47F0000E58EC2AF0AF
:1036C00061EC47F0000E58EC2AF061EC47F0000E78
:1036D00058EC2AF0E2EF1BF0D1EC46F0FF0E58EC6C
:1036E0002AF001EC46F0FF0E58EC2AF0E1EC46F02F
:1036F000FF0E58EC2AF0020E495CD8B487EF1BF09D
:10370000F1EC41F0FF0E58EC2AF08CEF1BF001ECCD
:1037100042F0FF0E58EC2AF061EC47F0000E58EC36
:103720002AF0E2EF1BF051EC46F0FF0E58EC2AF0C5
:1037300001EC47F0FF0E58EC2AF0E1EC46F0FF0EEA
:1037400058EC2AF0F1EC46F0FF0E58EC2AF061EC50
:1037500047F0000E58EC2AF0E2EF1BF0F1EC45F0D8
:10376000FF0E58EC2AF001EC46F0FF0E58EC2AF060
:1037700071EC46F0FF0E58EC2AF061EC47F0000EB9
:1037800058EC2AF061EC47F0000E58EC2AF0E2EF1A
:103790001BF0E1EC46F0FF0E58EC2AF0B1EC46F0DD
:1037A000FF0E58EC2AF0A1EC46F0FF0E58EC2AF080
:1037B00071EC46F0FF0E58EC2AF061EC47F0000E79
:1037C00058EC2AF03FB6E9EF1BF03F8616504A6EE0
:1037D0004B6E57EC31F01DEC2AF0400E26EC2AF02F
:1037E000BD0E3FEC2AF04050E8EC38F031EC39F0F7
:1037F0003F8274EF20F004EC3EF03FB202EF1CF089
:10380000070E496E3FA42EEC31F01AEC2AF0460E5A
:1038100026EC2AF0BC0E3FEC2AF0010E495CD8B42D
:1038200058EF1CF0020E495CD8B480EF1CF0030E78
:10383000495CD8B4A8EF1CF0040E495CD8B4D0EFB2
:103840001CF0050E495CD8B4F8EF1CF0060E495C7C
:10385000D8B420EF1DF0080E495CD8B446EF1DF037
:10386000FF0E58EC2AF0B1EC46F0FF0E58EC2AF0AF
:10387000C1EC45F0FF0E58EC2AF0D1EC46F0FF0EFB
:1038800058EC2AF081EC46F0FF0E58EC2AF061EC7F
:1038900047F0000E58EC2AF061EC47F0000E58ECAF
:1038A0002AF061EC47F0000E58EC2AF046EF1DF0CC
:1038B000FF0E58EC2AF0C1EC46F0FF0E58EC2AF04F
:1038C000E1EC45F0FF0E58EC2AF0D1EC46F0FF0E8B
:1038D00058EC2AF0E1EC45F0FF0E58EC2AF081ECB0
:1038E00046F0FF0E58EC2AF061EC47F0000E58EC61
:1038F0002AF061EC47F0000E58EC2AF046EF1DF07C
:10390000FF0E58EC2AF0E1EC45F0FF0E58EC2AF0DF
:10391000E1EC45F0FF0E58EC2AF0D1EC46F0FF0E3A
:1039200058EC2AF0E1EC45F0FF0E58EC2AF081EC5F
:1039300046F0FF0E58EC2AF061EC47F0000E58EC10
:103940002AF061EC47F0000E58EC2AF046EF1DF02B
:10395000FF0E58EC2AF001EC47F0FF0E58EC2AF06D
:1039600091EC46F0FF0E58EC2AF071EC46F0FF0E99
:1039700058EC2AF0A1EC46F0FF0E58EC2AF0E1ECEE
:1039800045F0FF0E58EC2AF061EC46F0FF0E58ECC3
:103990002AF081EC46F0FF0E58EC2AF046EF1DF0BD
:1039A000FF0E58EC2AF011EC47F0FF0E58EC2AF00D
:1039B00081EC46F0FF0E58EC2AF061EC47F0000E67
:1039C00058EC2AF061EC47F0000E58EC2AF061EC5C
:1039D00047F0000E58EC2AF061EC47F0000E58EC6E
:1039E0002AF061EC47F0000E58EC2AF046EF1DF08B
:1039F000FF0E58EC2AF0E1EC45F0FF0E58EC2AF0EF
:103A0000A1EC46F0FF0E58EC2AF081EC46F0FF0ED8
:103A100058EC2AF011EC46F0FF0E58EC2AF081EC3D
:103A200046F0FF0E58EC2AF061EC47F0000E58EC1F
:103A30002AF061EC47F0000E58EC2AF046EF1DF03A
:103A4000FF0E58EC2AF0D1EC45F0FF0E58EC2AF0AE
:103A500041EC46F0FF0E58EC2AF0B1EC46F0FF0EB8
:103A600058EC2AF081EC46F0FF0E58EC2AF061EC9D
:103A700047F0000E58EC2AF061EC47F0000E58ECCD
:103A80002AF061EC47F0000E58EC2AF03FB64DEFFB
:103A90001DF03F8617504A6E4B6E57EC31F01DEC0F
:103AA0002AF0400E26EC2AF0BD0E3FEC2AF04050E2
:103AB000E8EC38F031EC39F03F8274EF20F092EC12
:103AC0003EF03FB266EF1DF0070E496E3FA42EECAC
:103AD00031F01AEC2AF0460E26EC2AF0BC0E3FEC30
:103AE0002AF0010E495CD8B4A7EF1DF0020E495C24
:103AF000D8B4B5EF1DF0030E495CD8B4BEEF1DF08D
:103B0000040E495CD8B4CCEF1DF0050E495CD8B466
:103B1000DFEF1DF0060E495CD8B4EDEF1DF0080E86
:103B2000495CD8B4FEEF1DF09EEC40F081EC46F00D
:103B3000FF0E58EC2AF061EC47F0000E58EC2AF02A
:103B400061EC47F0000E58EC2AF0FEEF1DF013EC8C
:103B500040F081EC46F0FF0E58EC2AF061EC47F0A3
:103B6000000E58EC2AF0FEEF1DF02BEC40F081EC3B
:103B700046F0FF0E58EC2AF0FEEF1DF048EC40F046
:103B800081EC46F0FF0E58EC2AF061EC47F0000E95
:103B900058EC2AF0FEEF1DF060EC40F081EC46F0AE
:103BA000FF0E58EC2AF061EC47F0000E58EC2AF0BA
:103BB00061EC47F0000E58EC2AF0FEEF1DF073ECBC
:103BC00040F081EC46F0FF0E58EC2AF061EC47F033
:103BD000000E58EC2AF0FEEF1DF08BEC40F081EC6B
:103BE00046F0FF0E58EC2AF061EC47F0000E58EC5E
:103BF0002AF061EC47F0000E58EC2AF03FB605EFD2
:103C00001EF03F8618504A6E4B6E57EC31F01DEC9B
:103C10002AF0400E26EC2AF0BD0E3FEC2AF0405070
:103C2000E8EC38F031EC39F03F8274EF20F001EC31
:103C30003FF03FB21EEF1EF0070E496E3FA42EEC80
:103C400031F01AEC2AF0460E26EC2AF0BC0E3FECBE
:103C50002AF0010E495CD8B45FEF1EF0020E495CF9
:103C6000D8B46DEF1EF0030E495CD8B476EF1EF0A9
:103C7000040E495CD8B484EF1EF0050E495CD8B43C
:103C800097EF1EF0060E495CD8B4A5EF1EF0080EA3
:103C9000495CD8B4B6EF1EF09EEC40F001EC42F067
:103CA000FF0E58EC2AF061EC47F0000E58EC2AF0B9
:103CB00061EC47F0000E58EC2AF0B6EF1EF013EC62
:103CC00040F001EC42F0FF0E58EC2AF061EC47F0B6
:103CD000000E58EC2AF0B6EF1EF02BEC40F001EC91
:103CE00042F0FF0E58EC2AF0B6EF1EF048EC40F020
:103CF00001EC42F0FF0E58EC2AF061EC47F0000EA8
:103D000058EC2AF0B6EF1EF060EC40F001EC42F007
:103D1000FF0E58EC2AF061EC47F0000E58EC2AF048
:103D200061EC47F0000E58EC2AF0B6EF1EF073EC91
:103D300040F001EC42F0FF0E58EC2AF061EC47F045
:103D4000000E58EC2AF0B6EF1EF08BEC40F001ECC0
:103D500042F0FF0E58EC2AF061EC47F0000E58ECF0
:103D60002AF061EC47F0000E58EC2AF03FB6BDEFA8
:103D70001EF03F8619504A6E4B6E57EC31F01DEC29
:103D80002AF0400E26EC2AF0BD0E3FEC2AF04050FF
:103D9000E8EC38F031EC39F03F8274EF20F08AEC37
:103DA0003FF03FB2D6EF1EF0070E496E3FA42EEC57
:103DB00031F01AEC2AF0460E26EC2AF0BC0E3FEC4D
:103DC0002AF0010E495CD8B417EF1FF0020E495CCF
:103DD000D8B425EF1FF0030E495CD8B42EEF1FF0C6
:103DE000040E495CD8B43CEF1FF0050E495CD8B412
:103DF0004FEF1FF0060E495CD8B45DEF1FF0080EC0
:103E0000495CD8B46EEF1FF09EEC40F0F1EC41F04D
:103E1000FF0E58EC2AF061EC47F0000E58EC2AF047
:103E200061EC47F0000E58EC2AF06EEF1FF013EC37
:103E300040F0F1EC41F0FF0E58EC2AF061EC47F055
:103E4000000E58EC2AF06EEF1FF02BEC40F0F1EC76
:103E500041F0FF0E58EC2AF06EEF1FF048EC40F0F6
:103E6000F1EC41F0FF0E58EC2AF061EC47F0000E47
:103E700058EC2AF06EEF1FF060EC40F0F1EC41F0EE
:103E8000FF0E58EC2AF061EC47F0000E58EC2AF0D7
:103E900061EC47F0000E58EC2AF06EEF1FF073EC67
:103EA00040F0F1EC41F0FF0E58EC2AF061EC47F0E5
:103EB000000E58EC2AF06EEF1FF08BEC40F0F1ECA6
:103EC00041F0FF0E58EC2AF061EC47F0000E58EC80
:103ED0002AF061EC47F0000E58EC2AF03FB675EF7F
:103EE0001FF03F861A504A6E4B6E57EC31F01DECB6
:103EF0002AF0400E26EC2AF0BD0E3FEC2AF040508E
:103F0000E8EC38F031EC39F03F8274EF20F061ECEE
:103F100044F0000E58EC2AF071EC44F0000E58EC1E
:103F20002AF081EC44F0000E58EC2AF031EC44F019
:103F3000000E58EC2AF061EC45F0000E58EC2AF027
:103F4000D1EC44F0000E58EC2AF051EC45F0000E94
:103F500058EC2AF061EC47F0D1EC44F0000E58EC3C
:103F60002AF001EC45F01DEC2AF0400E26EC2AF078
:103F7000B90E3FEC2AF0000E58EC2AF031EC44F078
:103F8000000E58EC2AF061EC44F0000E58EC2AF0D8
:103F90001AEC2AF0670E26EC2AF0BC0E3FEC2AF051
:103FA0003FB0E7EF1FF0000E58EC2AF0A1EC45F00F
:103FB000000E58EC2AF071EC44F0000E58EC2AF098
:103FC00041EC45F0000E58EC2AF0F9EF1FF0FF0E1F
:103FD00058EC2AF041EC47F0FF0E58EC2AF001ECC7
:103FE00046F0FF0E58EC2AF0E1EC46F0FF0E58ECDC
:103FF0002AF01DEC2AF0440E26EC2AF0BC0E3FEC11
:104000002AF03FB018EF20F0FF0E58EC2AF091ECA8
:1040100046F0FF0E58EC2AF071EC47F0FF0E58EC1A
:104020002AF0A1EC46F0FF0E58EC2AF02AEF20F01F
:10403000000E58EC2AF0F1EC44F0000E58EC2AF097
:1040400061EC47F0000E58EC2AF001EC45F0000E50
:1040500058EC2AF080B03AEF20F03EB03BEF20F071
:104060003FB036EF20F03F8037EF20F03F903E80AA
:104070003BEF20F03E9084B64BEF20F03EBC4CEF7F
:1040800020F03FB047EF20F03F8048EF20F03F9016
:104090003E8C4CEF20F03E9C80B873EF20F03EB891
:1040A00074EF20F0436A466A42EC2BF03FA06FEFBA
:1040B00020F0080E116E040E126E4B0E136EBB0E26
:1040C000146E9B0E156E880E166E7F0E176E7F0E89
:1040D000186E000E196E000E1A6E5FEC2BF03F90FA
:1040E0003E881BEF01F03E9880BA87EF20F03EBA81
:1040F0001BEF01F0000E436E3E8A466A42EC2BF045
:104100003F903F923F96496A4A6A1BEF01F03E9A00
:104110001BEF01F01AEC2AF0410E26EC2AF0B80E43
:104120003FEC2AF0700E58EC2AF0100E58EC2AF0F2
:10413000100E58EC2AF0100E58EC2AF0000E58EC35
:104140002AF071EC44F0000E58EC2AF071EC44F0C7
:10415000000E58EC2AF011EC45F0000E58EC2AF055
:1041600031EC45F0000E58EC2AF001EC45F0000E61
:1041700058EC2AF0E1EC44F0000E58EC2AF061EC27
:1041800047F081EC45F0000E58EC2AF031EC45F098
:10419000000E58EC2AF0B1EC44F01DEC2AF0400E71
:1041A00026EC2AF0B80E3FEC2AF0000E58EC2AF06C
:1041B00051EC45F0000E58EC2AF071EC44F0000E82
:1041C00058EC2AF0082A320E085CD8B4EDEF20F043
:1041D000100E58EC2AF0E2EF20F0086A700E58EC4E
:1041E0002AF0000E445CD8B4FDEF20F0010E445CD0
:1041F000D8B487EF24F01BEF01F01AEC2AF0460E3A
:1042000026EC2AF0B90E3FEC2AF041EC45F0000E06
:1042100058EC2AF071EC44F0000E58EC2AF0D1EC86
:1042200044F0000E58EC2AF071EC44F0000E58EC0B
:104230002AF051EC44F0000E58EC2AF051EC45F015
:10424000000E58EC2AF061EC47F031EC44F0000E1F
:1042500058EC2AF061EC44F0000E58EC2AF061ECC6
:1042600044F01DEC2AF0400E26EC2AF0B90E3FEC8B
:104270002AF0000E58EC2AF031EC45F0000E58EC14
:104280002AF071EC44F0000E58EC2AF041EC45F0B5
:10429000000E58EC2AF041EC45F0000E58EC2AF0E4
:1042A00080B062EF21F03EB063EF21F00B0E475C6F
:1042B000D8B45EEF21F0472A5FEF21F0476A3E80D5
:1042C00063EF21F03E9084B676EF21F03EBC77EFAD
:1042D00021F0000E475CD8B471EF21F0470673EF70
:1042E00021F00B0E476E3E8C77EF21F03E9C1AECCE
:1042F0002AF04A0E26EC2AF0BB0E3FEC2AF0000E04
:10430000475CD8B498EF21F0000E58EC2AF051EC3D
:1043100041F0000E58EC2AF051EC41F0000E58EC40
:104320002AF0A1EC44F0000E58EC2AF0AAEF21F09C
:10433000FF0E58EC2AF0F1EC41F0FF0E58EC2AF099
:10434000F1EC41F0FF0E58EC2AF031EC46F0FF0E94
:1043500058EC2AF01AEC2AF0670E26EC2AF0BB0E75
:104360003FEC2AF0010E475CD8B4CBEF21F0000EF1
:1043700058EC2AF051EC41F0000E58EC2AF061ECB8
:1043800041F0000E58EC2AF0A1EC44F0000E58EC7D
:104390002AF0DDEF21F0FF0E58EC2AF0F1EC41F0AD
:1043A000FF0E58EC2AF001EC42F0FF0E58EC2AF018
:1043B00031EC46F0FF0E58EC2AF01DEC2AF0440ECA
:1043C00026EC2AF0BB0E3FEC2AF0020E475CD8B474
:1043D000FEEF21F0000E58EC2AF051EC41F0000EF7
:1043E00058EC2AF071EC41F0000E58EC2AF0A1ECE8
:1043F00044F0000E58EC2AF010EF22F0FF0E58ECBB
:104400002AF0F1EC41F0FF0E58EC2AF011EC42F0EA
:10441000FF0E58EC2AF031EC46F0FF0E58EC2AF073
:104420001DEC2AF0610E26EC2AF0BB0E3FEC2AF0C0
:10443000030E475CD8B431EF22F0000E58EC2AF09E
:1044400051EC41F0000E58EC2AF081EC41F0000EE6
:1044500058EC2AF0A1EC44F0000E58EC2AF043EF9F
:1044600022F0FF0E58EC2AF0F1EC41F0FF0E58EC70
:104470002AF021EC42F0FF0E58EC2AF031EC46F025
:10448000FF0E58EC2AF01AEC2AF04A0E26EC2AF01D
:10449000BC0E3FEC2AF0040E475CD8B464EF22F067
:1044A000000E58EC2AF051EC41F0000E58EC2AF0C6
:1044B00091EC41F0000E58EC2AF0A1EC44F0000E13
:1044C00058EC2AF076EF22F0FF0E58EC2AF0F1ECCF
:1044D00041F0FF0E58EC2AF031EC42F0FF0E58ECA0
:1044E0002AF031EC46F0FF0E58EC2AF01AEC2AF0D4
:1044F000670E26EC2AF0BC0E3FEC2AF0050E475C56
:10450000D8B497EF22F0000E58EC2AF051EC41F0AD
:10451000000E58EC2AF0A1EC41F0000E58EC2AF005
:10452000A1EC44F0000E58EC2AF0A9EF22F0FF0EA7
:1045300058EC2AF0F1EC41F0FF0E58EC2AF041EC77
:1045400042F0FF0E58EC2AF031EC46F0FF0E58EC2A
:104550002AF01DEC2AF0440E26EC2AF0BC0E3FECAB
:104560002AF0060E475CD8B4CAEF22F0000E58ECD1
:104570002AF051EC41F0000E58EC2AF0B1EC41F079
:10458000000E58EC2AF0A1EC44F0000E58EC2AF092
:10459000DCEF22F0FF0E58EC2AF0F1EC41F0FF0EB8
:1045A00058EC2AF051EC42F0FF0E58EC2AF031ECB6
:1045B00046F0FF0E58EC2AF01DEC2AF0610E26ECB6
:1045C0002AF0B40E3FEC2AF0070E475CD8B4FDEF9A
:1045D00022F0000E58EC2AF051EC41F0000E58EC9D
:1045E0002AF0C1EC41F0000E58EC2AF0A1EC44F0A6
:1045F000000E58EC2AF00FEF23F0FF0E58EC2AF0D3
:10460000F1EC41F0FF0E58EC2AF061EC42F0FF0EA5
:1046100058EC2AF031EC46F0FF0E58EC2AF01AEC78
:104620002AF04A0E26EC2AF0BD0E3FEC2AF0080EC6
:10463000475CD8B430EF23F0000E58EC2AF051EC70
:1046400041F0000E58EC2AF0D1EC41F0000E58EC8D
:104650002AF0A1EC44F0000E58EC2AF042EF23F0CF
:10466000FF0E58EC2AF0F1EC41F0FF0E58EC2AF066
:1046700071EC42F0FF0E58EC2AF031EC46F0FF0EE0
:1046800058EC2AF01AEC2AF0670E26EC2AF0BD0E40
:104690003FEC2AF0090E475CD8B463EF23F0000E1C
:1046A00058EC2AF051EC41F0000E58EC2AF0E1EC05
:1046B00041F0000E58EC2AF0A1EC44F0000E58EC4A
:1046C0002AF075EF23F0FF0E58EC2AF0F1EC41F0E0
:1046D000FF0E58EC2AF081EC42F0FF0E58EC2AF065
:1046E00031EC46F0FF0E58EC2AF01AEC2AF04A0E94
:1046F00026EC2AF0BE0E3FEC2AF00A0E475CD8B436
:10470000B1EF23F0000E58EC2AF001EC45F0000E5A
:1047100058EC2AF051EC45F0000E58EC2AF0A1ECD0
:1047200044F0000E58EC2AF071EC44F0000E58EC06
:104730002AF031EC45F0000E58EC2AF061EC47F01D
:1047400041EC45F0000E58EC2AF071EC44F0000EFC
:1047500058EC2AF051EC45F0000E58EC2AF0DEEF50
:1047600023F0FF0E58EC2AF0A1EC46F0FF0E58ECB7
:104770002AF0F1EC46F0FF0E58EC2AF031EC46F04E
:10478000FF0E58EC2AF001EC46F0FF0E58EC2AF030
:10479000D1EC46F0FF0E58EC2AF071EC47F0E1EC5A
:1047A00046F0FF0E58EC2AF001EC46F0FF0E58ECF4
:1047B0002AF0F1EC46F0FF0E58EC2AF01AEC2AF041
:1047C0004A0E26EC2AF0BF0E3FEC2AF00B0E475C97
:1047D000D8B431EF24F0000E58EC2AF031EC44F05C
:1047E000000E58EC2AF0D1EC44F0000E58EC2AF000
:1047F000D1EC44F0000E58EC2AF061EC47F031ECBB
:1048000045F0000E58EC2AF071EC44F0000E58EC24
:104810002AF091EC44F0000E58EC2AF0B1EC44F090
:10482000000E58EC2AF041EC45F0000E58EC2AF04E
:104830001DEC2AF0400E26EC2AF0BF0E3FEC2AF0C9
:1048400051EC45F0000E58EC2AF071EC44F0000EEB
:1048500058EC2AF031EC45F0000E58EC2AF075EFD8
:1048600024F0FF0E58EC2AF0C1EC45F0FF0E58EC96
:104870002AF071EC46F0FF0E58EC2AF071EC46F08D
:10488000FF0E58EC2AF071EC47F0D1EC46F0FF0E29
:1048900058EC2AF001EC46F0FF0E58EC2AF021EC1F
:1048A00046F0FF0E58EC2AF041EC46F0FF0E58ECB3
:1048B0002AF0E1EC46F0FF0E58EC2AF01DEC2AF04D
:1048C000400E26EC2AF0BF0E3FEC2AF0F1EC46F049
:1048D000FF0E58EC2AF001EC46F0FF0E58EC2AF0DF
:1048E000D1EC46F0FF0E58EC2AF0DBEC2DF080B84E
:1048F00084EF24F03EB885EF24F0010E446E42ECC4
:104900002BF03E8885EF24F03E981BEF01F01AEC67
:104910002AF0460E26EC2AF0B90E3FEC2AF0000EE3
:10492000475CD8B4C8EF24F0010E475CD8B4D0EF90
:1049300024F0020E475CD8B4D8EF24F0030E475C95
:10494000D8B4E0EF24F0040E475CD8B4E8EF24F0CC
:10495000050E475CD8B4F0EF24F0060E475CD8B4DF
:10496000F8EF24F0070E475CD8B400EF25F0080EEE
:10497000475CD8B408EF25F0090E475CD8B410EFB7
:1049800025F00A0E475CD8B418EF25F072EF25F039
:104990009EEC3BF0AEEC33F033EC34F0F9EF25F065
:1049A000F7EC3BF0AEEC33F033EC34F0F9EF25F0FC
:1049B00050EC3CF0AEEC33F033EC34F0F9EF25F092
:1049C000A9EC3CF0AEEC33F033EC34F0F9EF25F029
:1049D00002EC3DF0AEEC33F033EC34F0F9EF25F0BF
:1049E0005BEC3DF0AEEC33F033EC34F0F9EF25F056
:1049F00004EC3EF0AEEC33F033EC34F0F9EF25F09C
:104A000092EC3EF0AEEC33F033EC34F0F9EF25F0FD
:104A100001EC3FF0AEEC33F033EC34F0F9EF25F07D
:104A20008AEC3FF0AEEC33F033EC34F0F9EF25F0E4
:104A3000000E58EC2AF001EC45F0000E58EC2AF07C
:104A400051EC45F0000E58EC2AF0A1EC44F0000EB9
:104A500058EC2AF071EC44F0000E58EC2AF031ECDE
:104A600045F0000E58EC2AF061EC47F041EC45F0BF
:104A7000000E58EC2AF071EC44F0000E58EC2AF0CD
:104A800051EC45F0000E58EC2AF01DEC2AF0400ED7
:104A900026EC2AF0B90E3FEC2AF0000E58EC2AF072
:104AA000000E58EC2AF081EC45F0000E58EC2AF08C
:104AB00031EC45F0000E58EC2AF0B1EC44F0000E59
:104AC00058EC2AF051EC45F0000E58EC2AF071EC4D
:104AD00044F0000E58EC2AF0AEEC33F033EC34F036
:104AE000F9EF25F031EC44F0000E58EC2AF0D1EC4F
:104AF00044F0000E58EC2AF0D1EC44F0000E58ECD3
:104B00002AF061EC47F031EC45F0000E58EC2AF049
:104B100071EC44F0000E58EC2AF091EC44F0000ED9
:104B200058EC2AF0B1EC44F0000E58EC2AF041ECBD
:104B300045F0000E58EC2AF051EC45F01DEC2AF03F
:104B4000400E26EC2AF0B90E3FEC2AF0000E58EC8D
:104B50002AF071EC44F0000E58EC2AF031EC45F0EC
:104B6000000E58EC2AF061EC47F081EC45F0000EA5
:104B700058EC2AF031EC45F0000E58EC2AF0B1EC7C
:104B800044F0000E58EC2AF051EC45F0000E58ECC1
:104B90002AF071EC44F0000E58EC2AF0AEEC33F041
:104BA00080B8F8EF25F03EB8F9EF25F03FACF1EF13
:104BB00025F042EC2BF099EC47F0ACEC47F0BFEC61
:104BC00047F0D2EC47F0E5EC47F0F8EC47F00BEC9F
:104BD00048F01EEC48F031EC48F044EC48F057EC5B
:104BE00048F0446A476A3F9C3F903E881BEF01F0C3
:104BF0003E9880BA1BEF01F0000E446E3E8A476A71
:104C000042EC2BF03F9C1BEF01F01AEC2AF0410E16
:104C100026EC2AF0B80E3FEC2AF0700E58EC2AF081
:104C2000100E58EC2AF0100E58EC2AF0100E58EC2A
:104C30002AF0000E58EC2AF001EC45F0000E58EC7A
:104C40002AF051EC45F0000E58EC2AF0A1EC44F0AB
:104C5000000E58EC2AF071EC44F0000E58EC2AF0EB
:104C600031EC45F0000E58EC2AF061EC47F041ECD5
:104C700045F0000E58EC2AF071EC44F0000E58ECB0
:104C80002AF051EC45F0000E58EC2AF051EC45F0BA
:104C90001DEC2AF0400E26EC2AF0B80E3FEC2AF06C
:104CA000000E58EC2AF0B1EC44F0000E58EC2AF05B
:104CB000F1EC44F0000E58EC2AF091EC44F0000EB8
:104CC00058EC2AF0082A2C0E085CD8B46DEF26F0B8
:104CD000100E58EC2AF062EF26F0086A700E58ECBD
:104CE0002AF01AEC2AF0460E26EC2AF0BF0E3FEC12
:104CF0002AF041EC45F0000E58EC2AF001EC45F0AA
:104D0000000E58EC2AF081EC44F0000E58EC2AF02A
:104D100051EC45F0000E58EC2AF081EC45F0000E05
:104D200058EC2AF031EC44F0000E58EC2AF031EC4B
:104D300045F0000E58EC2AF071EC44F0000E58ECEF
:104D40002AF061EC47F071EC45F01DEC2AF0400EC2
:104D500026EC2AF0BF0E3FEC2AF0000E58EC2AF0A9
:104D600071EC44F0000E58EC2AF031EC45F0000EE6
:104D700058EC2AF041EC45F0000E58EC2AF0B1EC6A
:104D800044F0000E58EC2AF001EC45F0000E58EC0F
:104D90002AF0F1EC44F0000E58EC2AF061EC47F0F8
:104DA000000E58EC2AF061EC41F0000E58EC2AF0AD
:104DB000000E58EC2AF0400E58EC2AF0000E58EC89
:104DC0002AF051EC41F0000E58EC2AF081EC41F051
:104DD000000E58EC2AF01AEC2AF0450E26EC2AF0C8
:104DE000BA0E3FEC2AF04CBE37EF27F0000E485CBD
:104DF000D8A437EF27F0FF0E58EC2AF001EC46F06C
:104E0000FF0E58EC2AF0D1EC46F0FF0E58EC2AF0D9
:104E1000D1EC46F0FF0E58EC2AF0A1EC46F0FF0E64
:104E200058EC2AF0D1EC46F0FF0E58EC2AF071EC69
:104E300047F031EC46F0FF0E58EC2AF0A1EC46F0BA
:104E4000FF0E58EC2AF071EC46F0FF0E58EC2AF0F9
:104E5000F1EC45F01DEC2AF0400E26EC2AF0BA0EDB
:104E60003FEC2AF0FF0E58EC2AF071EF27F0000E0D
:104E700058EC2AF071EC44F0000E58EC2AF031ECBA
:104E800045F0000E58EC2AF031EC45F0000E58ECDD
:104E90002AF001EC45F0000E58EC2AF031EC45F018
:104EA000000E58EC2AF061EC47F0A1EC44F0000E43
:104EB00058EC2AF001EC45F0000E58EC2AF0D1EC49
:104EC00044F0000E58EC2AF061EC44F01DEC2AF09E
:104ED000400E26EC2AF0BA0E3FEC2AF0000E58ECF9
:104EE0002AF01AEC2AF0450E26EC2AF0BB0E3FEC15
:104EF0002AF04CBEB0EF27F0010E485CD8A4B0EF0A
:104F000027F0FF0E58EC2AF0F1EC46F0FF0E58ECBB
:104F10002AF031EC47F0FF0E58EC2AF071EC47F024
:104F2000A1EC46F0FF0E58EC2AF001EC47F0FF0E22
:104F300058EC2AF0F1EC46F0FF0E58EC2AF0B1ECF8
:104F400046F0FF0E58EC2AF001EC47F0FF0E58EC4B
:104F50002AF0F1EC46F0FF0E58EC2AF0DDEF27F0D6
:104F6000000E58EC2AF051EC45F0000E58EC2AF0F7
:104F700091EC45F0000E58EC2AF061EC47F001ECA2
:104F800045F0000E58EC2AF061EC45F0000E58ECAC
:104F90002AF051EC45F0000E58EC2AF011EC45F0E7
:104FA000000E58EC2AF061EC45F0000E58EC2AF0A7
:104FB00051EC45F0000E58EC2AF01AEC2AF0450EA0
:104FC00026EC2AF0BC0E3FEC2AF04CBE29EF28F06C
:104FD000020E485CD8A429EF28F0FF0E58EC2AF006
:104FE000E1EC46F0FF0E58EC2AF001EC46F0FF0E23
:104FF00058EC2AF071EC46F0FF0E58EC2AF001EC68
:1050000046F0FF0E58EC2AF0E1EC45F0FF0E58ECAC
:105010002AF0F1EC46F0FF0E58EC2AF071EC47F064
:1050200001EC47F0FF0E58EC2AF0E1EC46F0FF0EE1
:1050300058EC2AF0D1EC45F01DEC2AF0400E26EC9D
:105040002AF0BC0E3FEC2AF0FF0E58EC2AF063EF7A
:1050500028F0000E58EC2AF041EC45F0000E58EC18
:105060002AF071EC44F0000E58EC2AF0D1EC44F038
:10507000000E58EC2AF071EC44F0000E58EC2AF0C7
:1050800051EC44F0000E58EC2AF051EC45F0000EC3
:1050900058EC2AF061EC47F061EC45F0000E58EC5A
:1050A0002AF041EC45F0000E58EC2AF041EC44F0B7
:1050B0001DEC2AF0400E26EC2AF0BC0E3FEC2AF044
:1050C000000E58EC2AF04CBE8DEF28F080B078EF3F
:1050D00028F03EB079EF28F0020E485CD8B474EFA7
:1050E00028F0482A75EF28F0486A3E8079EF28F0CA
:1050F0003E9084B68CEF28F03EBC8DEF28F0000E79
:10510000485CD8B487EF28F0480689EF28F0020EF3
:10511000486E3E8C8DEF28F03E9C4CBE9DEF28F0F3
:1051200080B89CEF28F03EB89DEF28F04C8E4C5094
:105130004D6E3E889DEF28F03E984CAEADEF28F0C6
:1051400080BAACEF28F03EBAADEF28F04C9E42ECAE
:105150002BF03E8AADEF28F03E9A4CAEBFEF28F020
:1051600080B8BEEF28F03EB8BFEF28F04D504C6E2F
:105170004C9E42EC2BF03E88BFEF28F03E984CAEA0
:1051800006EF29F080B0E3EF28F03EB0E4EF28F01E
:10519000000E485CD8B4D9EF28F0010E485CD8B4B2
:1051A000DCEF28F0020E485CD8B4DFEF28F0E0EF27
:1051B00028F04D70E0EF28F04D72E0EF28F04D74CC
:1051C0003E80E4EF28F03E9084B605EF29F03EBC27
:1051D00006EF29F0000E485CD8B4FBEF28F0010E72
:1051E000485CD8B4FEEF28F0020E485CD8B401EF5A
:1051F00029F002EF29F04D7002EF29F04D7202EF15
:1052000029F04D743E8C06EF29F03E9C4CAE15EF14
:105210002AF0000E485CD8B41AEF29F0010E485C61
:10522000D8B457EF29F0020E485CD8B4C6EF29F085
:1052300015EF2AF01DEC2AF0460E26EC2AF0BA0EE5
:105240003FEC2AF04DA03EEF29F0FF0E58EC2AF07B
:1052500031EC46F0FF0E58EC2AF0A1EC46F0FF0EC0
:1052600058EC2AF071EC46F0FF0E58EC2AF0F1EC05
:1052700045F0FF0E58EC2AF015EF2AF0FF0E58EC1F
:105280002AF011EC46F0FF0E58EC2AF0D1EC46F073
:10529000FF0E58EC2AF001EC46F0FF0E58EC2AF015
:1052A00001EC46F0FF0E58EC2AF015EF2AF01DEC49
:1052B0002AF0460E26EC2AF0BB0E3FEC2AF04DA257
:1052C00094EF29F0FF0E58EC2AF041EC46F0FF0E67
:1052D00058EC2AF091EC46F0FF0E58EC2AF0F1EC75
:1052E00046F0FF0E58EC2AF001EC46F0FF0E58ECA9
:1052F0002AF0D1EC46F0FF0E58EC2AF071EC46F0A3
:10530000FF0E58EC2AF0A1EC46F0FF0E58EC2AF004
:10531000E1EC45F0FF0E58EC2AF061EC46F0FF0E90
:1053200058EC2AF015EF2AF0FF0E58EC2AF011EC99
:1053300046F0FF0E58EC2AF0D1EC46F0FF0E58EC88
:105340002AF001EC46F0FF0E58EC2AF001EC46F092
:10535000FF0E58EC2AF061EC47F0000E58EC2AF0F2
:1053600061EC47F0000E58EC2AF061EC47F0000EBB
:1053700058EC2AF061EC47F0000E58EC2AF061EC92
:1053800047F0000E58EC2AF015EF2AF01DEC2AF039
:10539000460E26EC2AF0BC0E3FEC2AF04DA4F4EFAA
:1053A00029F0FF0E58EC2AF0C1EC45F0FF0E58EC46
:1053B0002AF001EC47F0FF0E58EC2AF0F1EC46F031
:1053C000FF0E58EC2AF0A1EC46F0FF0E58EC2AF044
:1053D00061EC47F0000E58EC2AF061EC47F0000E4B
:1053E00058EC2AF015EF2AF0FF0E58EC2AF081EC69
:1053F00046F0FF0E58EC2AF0C1EC45F0FF0E58ECD9
:105400002AF091EC46F0FF0E58EC2AF001EC47F040
:10541000FF0E58EC2AF0C1EC45F0FF0E58EC2AF0D4
:1054200071EC46F0FF0E58EC2AF04CAEDBEC2DF0A0
:105430001BEF01F08C888B9E12008C988B8E1200D3
:105440008C888B8E12008C988B9E1200016E1FEC44
:105450002BF001508A6E8C9C8C9E000000008C8A80
:10546000000000000000000000000000000000003C
:105470008C9A000000000000000000001200026E84
:105480001FEC2BF002508A6E8C9C8C9E000000005A
:105490008C8A0000000000000000000000000000F6
:1054A00000008C9A000000000000000000001200C4
:1054B000006E1FEC2BF03FBE74EC2AF000508A6E99
:1054C0008C9C8C8E000000008C8A00000000000084
:1054D000000000000000000000008C9A00000000A6
:1054E0000000000000001200000E515CD8B499EFDB
:1054F0002AF0010E515CD8B4B2EF2AF0020E515CD2
:10550000D8B4C9EF2AF0030E515CD8B4DEEF2AF00C
:10551000040E515CD8B4F1EF2AF0050E515CD8B4FA
:1055200002EF2BF0060E515CD8B411EF2BF01EEFFA
:105530002BF050B0A7EF2AF0004200420042004298
:10554000004200420042010E00161EEF2BF0004602
:10555000004600460046004600460046800E001603
:105560001EEF2BF050B0BFEF2AF000420042004285
:10557000004200420042030E00161EEF2BF00046D0
:1055800000460046004600460046C00E00161EEFCC
:105590002BF050B0D5EF2AF000420042004200420A
:1055A0000042070E00161EEF2BF000460046004694
:1055B00000460046E00E00161EEF2BF050B0E9EF5B
:1055C0002AF000420042004200420F0E00161EEF79
:1055D0002BF00046004600460046F00E00161EEF77
:1055E0002BF050B0FBEF2AF00042004200421F0EA9
:1055F00000161EEF2BF0004600460046F80E00167F
:105600001EEF2BF050B00BEF2BF0004200423F0E8C
:1056100000161EEF2BF000460046FC0E00161EEF93
:105620002BF050B019EF2BF000427F0E00161EEF4A
:105630002BF00046FE0E00161EEF2BF012000F019D
:10564000FF0E936E00018C8C8C9E000000008C8AF3
:10565000000000000000000000000000000000004A
:105660008C9A000000000000000000000000000014
:10567000000081BE27EF2BF08C9C0F01000E936E73
:105680000001120020EC2AF0400E26EC2AF0B80EA1
:105690003FEC2AF0000E58EC2AF0012A800E015C43
:1056A000D8A44AEF2BF0022A40EC2AF0400E26EC58
:1056B0002AF0C00E025CD8A44AEF2BF012008B80B7
:1056C00000008B92DBEC35F08B82DBEC35F07CEC70
:1056D0002BF092EC2BF0A7EC2BF0BCEC2BF0D1ECE8
:1056E0002BF0E6EC2BF0FBEC2BF010EC2CF025EC87
:1056F0002CF03AEC2CF012008B9000004FEC2CF0C8
:105700008B9400008B8600008B960000000E386E94
:105710007AEC2CF011503C6E8FEC2CF08B948B9625
:105720008B8012008B904FEC2CF08B9400008B86BA
:1057300000008B960000010E386E7AEC2CF01250AF
:105740003C6E8FEC2CF08B948B968B8012008B90A0
:105750004FEC2CF08B9400008B8600008B960000A1
:10576000020E386E7AEC2CF013503C6E8FEC2CF05D
:105770008B948B968B8012008B904FEC2CF08B943B
:1057800000008B8600008B960000030E386E7AECCA
:105790002CF014503C6E8FEC2CF08B948B968B80FD
:1057A00012008B904FEC2CF08B9400008B86000045
:1057B0008B960000040E386E7AEC2CF015503C6E7F
:1057C0008FEC2CF08B948B968B8012008B904FEC8F
:1057D0002CF08B9400008B8600008B960000050E49
:1057E000386E7AEC2CF016503C6E8FEC2CF08B94CB
:1057F0008B968B8012008B904FEC2CF08B940000DA
:105800008B8600008B960000060E386E7AEC2CF02A
:1058100017503C6E8FEC2CF08B948B968B80120083
:105820008B904FEC2CF08B9400008B8600008B96B5
:105830000000070E386E7AEC2CF018503C6E8FEC9E
:105840002CF08B948B968B8012008B904FEC2CF06D
:105850008B9400008B8600008B960000080E386E3B
:105860007AEC2CF019503C6E8FEC2CF08B948B96CC
:105870008B8012008B904FEC2CF08B9400008B8669
:1058800000008B960000090E386E7AEC2CF01A504E
:105890003C6E8FEC2CF08B948B968B8012008B944B
:1058A00000008B8600008B9600008B9400008B8696
:1058B00000008B9600008B8400008B8600008B9686
:1058C00000008B9400008B8600008B9600008B9468
:1058D00000008B8600008B9600008B9400008B8666
:1058E00000008B9600008B9400008B8600008B9646
:1058F0000000120038BE80EF2CF08B9482EF2CF069
:105900008B8400008B8600008B960000392A384675
:10591000080E395CD8A47AEF2CF0396A12003CBE2C
:1059200095EF2CF08B9497EF2CF08B8400008B86F6
:1059300000008B9600003A2A3C46080E3A5CD8A438
:105940008FEF2CF03A6A12008B904FEC2CF08B9476
:1059500000008B8600008B9600000A0E386E7AECF1
:105960002CF08B800000000000008B904FEC2CF09E
:105970008B8400008B8600008B96000000000000E6
:105980000000C7EC2CF08B948B968B8012008B86DA
:1059900083A0CEEF2CF03B80CFEF2CF03B903A2A47
:1059A0008B96080E3A5CD8B4D9EF2CF03B46C7EF83
:1059B0002CF03A6A3D2A010E3D5CD8A4E4EF2CF0AD
:1059C0003B501B6EC7EF2CF0020E3D5CD8A4EDEFF0
:1059D0002CF03B501C6EC7EF2CF0030E3D5CD8A49E
:1059E000F6EF2CF03B501D6EC7EF2CF0040E3D5C23
:1059F000D8A4FFEF2CF03B501E6EC7EF2CF0050E25
:105A00003D5CD8A408EF2DF03B501F6EC7EF2CF083
:105A1000060E3D5CD8A411EF2DF03B50206EC7EF71
:105A20002CF0070E3D5CD8A41AEF2DF03B50216EF0
:105A3000C7EF2CF0080E3D5CD8A423EF2DF03B50AF
:105A4000226EC7EF2CF0090E3D5CD8A42CEF2DF090
:105A50003B50236EC7EF2CF00A0E3D5CD8A435EF07
:105A60002DF03B50246EC7EF2CF00B0E3D5CD8A4FC
:105A70003EEF2DF03B50256EC7EF2CF00C0E3D5C39
:105A8000D8A447EF2DF03B50266EC7EF2CF00D0E3B
:105A90003D5CD8A450EF2DF03B50276EC7EF2CF0A3
:105AA0000E0E3D5CD8A459EF2DF03B50286EC7EF89
:105AB0002CF00F0E3D5CD8A462EF2DF03B50296E08
:105AC000C7EF2CF0100E3D5CD8A46BEF2DF03B50CF
:105AD0002A6EC7EF2CF0110E3D5CD8A474EF2DF0A8
:105AE0003B502B6EC7EF2CF0120E3D5CD8A47DEF1F
:105AF0002DF03B502C6EC7EF2CF0130E3D5CD8A45C
:105B000086EF2DF03B502D6EC7EF2CF0140E3D5C50
:105B1000D8A48FEF2DF03B502E6EC7EF2CF0150E52
:105B20003D5CD8A498EF2DF03B502F6EC7EF2CF0C2
:105B3000160E3D5CD8A4A1EF2DF03B50306EC7EFA0
:105B40002CF0170E3D5CD8A4AAEF2DF03B50316E1F
:105B5000C7EF2CF0180E3D5CD8A4B3EF2DF03B50EE
:105B6000326EC7EF2CF0190E3D5CD8A4BCEF2DF0BF
:105B70003B50336EC7EF2CF01A0E3D5CD8A4C5EF36
:105B80002DF03B50346EC7EF2CF01B0E3D5CD8A4BB
:105B9000CEEF2DF03B50356EC7EF2CF01C0E3D5C68
:105BA000D8A4D7EF2DF03B50366EC7EF2CF03B500A
:105BB000376E3D6A120080BAE8EF2DF03EBA12004F
:105BC00042EC2BF0416A466A476A486A3E8A1200F4
:105BD0003E9A1200000E405CD8A413EF2EF091EC18
:105BE00044F0000E58EC2AF0F1EC44F0000E58ECB2
:105BF0002AF061EC44F0000E58EC2AF061EC47F01A
:105C0000000E58EC2AF061EC47F0000E58EC2AF038
:105C100061EC47F0000E58EC2AF061EC47F0000E02
:105C200058EC2AF01200010E405CD8A43CEF2EF094
:105C300071EC44F0000E58EC2AF0E1EC44F0000E58
:105C400058EC2AF011EC45F0000E58EC2AF0A1ECCB
:105C500044F0000E58EC2AF061EC47F0000E58ECCE
:105C60002AF061EC47F0000E58EC2AF061EC47F0A6
:105C7000000E58EC2AF01200020E405CD8A465EF2A
:105C80002EF0B1EC44F0000E58EC2AF0F1EC44F0A8
:105C9000000E58EC2AF051EC45F0000E58EC2AF0BA
:105CA00061EC47F0000E58EC2AF061EC47F0000E72
:105CB00058EC2AF061EC47F0000E58EC2AF061EC49
:105CC00047F0000E58EC2AF01200030E405CD8A4F6
:105CD0008EEF2EF051EC44F0000E58EC2AF061ECFF
:105CE00047F0000E58EC2AF041EC45F0000E58EC5D
:105CF0002AF051EC45F0000E58EC2AF031EC44F05B
:105D0000000E58EC2AF061EC47F0000E58EC2AF037
:105D100061EC47F0000E58EC2AF01200040E405CD3
:105D2000D8A4B7EF2EF061EC45F0000E58EC2AF045
:105D300061EC47F0000E58EC2AF061EC44F0000EE4
:105D400058EC2AF031EC44F0000E58EC2AF051ECFB
:105D500045F0000E58EC2AF031EC44F0000E58ECFF
:105D60002AF061EC47F0000E58EC2AF01200050E04
:105D7000405CD8A4E0EF2EF031EC45F0000E58EC7A
:105D80002AF061EC47F0000E58EC2AF071EC44F078
:105D9000000E58EC2AF031EC45F0000E58EC2AF0D9
:105DA00031EC45F0000E58EC2AF061EC47F0000EA3
:105DB00058EC2AF061EC47F0000E58EC2AF0120083
:105DC000060E405CD8A409EF2FF0F1EC44F0000E71
:105DD00058EC2AF071EC45F0000E58EC2AF061EC1A
:105DE00047F0000E58EC2AF071EC44F0000E58EC2D
:105DF0002AF031EC45F0000E58EC2AF031EC45F079
:105E0000000E58EC2AF061EC47F0000E58EC2AF036
:105E10001200070E405CD8A432EF2FF031EC45F0B1
:105E2000000E58EC2AF051EC44F0000E58EC2AF029
:105E300041EC44F0000E58EC2AF0D1EC44F0000E96
:105E400058EC2AF061EC47F0000E58EC2AF061ECB7
:105E500047F0000E58EC2AF061EC47F0000E58ECC9
:105E60002AF01200080E405CD8A45BEF2FF0E1ECA2
:105E700041F0000E58EC2AF0B1EC41F0000E58EC65
:105E80002AF0C1EC44F0000E58EC2AF0A1EC44F0EA
:105E9000000E58EC2AF0B1EC45F0000E58EC2AF058
:105EA00061EC47F0000E58EC2AF061EC47F0000E70
:105EB00058EC2AF01200090E405CD8A484EF2FF0B1
:105EC00031EC44F0000E58EC2AF061EC45F0000E85
:105ED00058EC2AF061EC44F0000E58EC2AF0B1ECDA
:105EE00044F0000E58EC2AF001EC45F0000E58EC9E
:105EF0002AF061EC47F0000E58EC2AF061EC47F014
:105F0000000E58EC2AF012000A0E405CD8A4ADEF47
:105F10002FF071EC45F0000E58EC2AF0D1EC44F073
:105F2000000E58EC2AF031EC45F0000E58EC2AF047
:105F300051EC44F0000E58EC2AF0C1EC44F0000E95
:105F400058EC2AF061EC47F0000E58EC2AF061ECB6
:105F500047F0000E58EC2AF012000B0E405CD8A45B
:105F60008FEF30F051EC45F0000E58EC2AF091EC38
:105F700045F0000E58EC2AF061EC47F0000E58ECAA
:105F80002AF01550070B406E000E405CD8A4DEEFDF
:105F90002FF031EC45F0000E58EC2AF091EC45F072
:105FA000000E58EC2AF011EC45F0000E58EC2AF0E7
:105FB00051EC41F0000E58EC2AF01200010E405C4A
:105FC000D8A4F8EF2FF031EC45F0000E58EC2AF091
:105FD00091EC45F0000E58EC2AF011EC45F0000E63
:105FE00058EC2AF061EC41F0000E58EC2AF0120057
:105FF000020E405CD8A412EF30F031EC45F0000EF8
:1060000058EC2AF091EC45F0000E58EC2AF011EC17
:1060100045F0000E58EC2AF071EC41F0000E58ECFF
:106020002AF01200030E405CD8A42CEF30F061EC93
:1060300045F0000E58EC2AF041EC45F0000E58EC0B
:106040002AF041EC44F0000E58EC2AF061EC47F0E5
:10605000000E58EC2AF01200040E405CD8A446EF63
:1060600030F031EC45F0000E58EC2AF091EC45F0A0
:10607000000E58EC2AF011EC45F0000E58EC2AF016
:1060800091EC41F0000E58EC2AF01200050E405C35
:10609000D8A460EF30F031EC45F0000E58EC2AF057
:1060A00091EC45F0000E58EC2AF011EC45F0000E92
:1060B00058EC2AF0A1EC41F0000E58EC2AF0120046
:1060C000060E405CD8A47AEF30F031EC45F0000EBB
:1060D00058EC2AF091EC45F0000E58EC2AF011EC47
:1060E00045F0000E58EC2AF0B1EC41F0000E58ECEF
:1060F0002AF0120031EC45F0000E58EC2AF091EC39
:1061000045F0000E58EC2AF011EC45F0000E58EC6A
:106110002AF0C1EC41F0000E58EC2AF012000C0EEF
:10612000405CD8A4B8EF30F071EC45F0000E58ECAC
:106130002AF061EC44F0000E58EC2AF061EC44F0D7
:10614000000E58EC2AF061EC47F0000E58EC2AF0F3
:1061500061EC47F0000E58EC2AF061EC47F0000EBD
:1061600058EC2AF061EC47F0000E58EC2AF01200CF
:106170000D0E405CD8A4E1EF30F0A1EC44F0000E2D
:1061800058EC2AF031EC45F0000E58EC2AF0E1EC26
:1061900044F0000E58EC2AF051EC44F0000E58EC9C
:1061A0002AF0C1EC44F0000E58EC2AF061EC47F004
:1061B000000E58EC2AF061EC47F0000E58EC2AF083
:1061C000120031EC45F0000E58EC2AF071EC44F06E
:1061D000000E58EC2AF041EC45F0000E58EC2AF085
:1061E00071EC44F0000E58EC2AF031EC45F0000E52
:1061F00058EC2AF071EC45F0000E58EC2AF071ECE6
:1062000044F0000E58EC2AF0120080B018EF31F084
:106210003EB019EF31F0000E495CD8A414EF31F014
:10622000080E496E15EF31F049063E8019EF31F046
:106230003E9084B62CEF31F03EBC2DEF31F0080ECD
:10624000495CD8A428EF31F0000E496E29EF31F0F7
:10625000492A3E8C2DEF31F03E9C120080B041EF78
:1062600031F03EB042EF31F0010E495CD8A43DEF71
:1062700031F0080E496E3EEF31F049063E8042EFA4
:1062800031F03E9084B655EF31F03EBC56EF31F020
:10629000080E495CD8A451EF31F0010E496E52EF5F
:1062A00031F0492A3E8C56EF31F03E9C1200080E28
:1062B000495CD8B43BEF33F03FB493EF31F080B892
:1062C00069EF31F03EB826EF32F03F843E8893EF1D
:1062D00031F03E981AEC2AF04D0E26EC2AF0BE0E54
:1062E0003FEC2AF0000E58EC2AF061EC47F0000E6B
:1062F00058EC2AF061EC47F061EC47F0000E58ECE6
:106300002AF061EC47F0000E58EC2AF061EC47F0FF
:10631000000E58EC2AF061EC47F0000E58EC2AF021
:106320004A50406E12001AEC2AF04D0E26EC2AF06C
:10633000BE0E3FEC2AF0000E495CD8B4C0EF31F03D
:10634000010E495CD8B4C5EF31F0020E495CD8B4F7
:10635000CAEF31F0030E495CD8B4CFEF31F0040E30
:10636000495CD8B4D4EF31F0050E495CD8B4D9EF0C
:1063700031F0060E495CD8B4DEEF31F0E3EF31F0D6
:106380004BAEE8EF31F008EF32F04BACE8EF31F014
:1063900008EF32F04BAAE8EF31F008EF32F04BA8EB
:1063A000E8EF31F008EF32F04BA6E8EF31F008EFFC
:1063B00032F04BA4E8EF31F008EF32F04BA2E8EFF7
:1063C00031F008EF32F04BA0E8EF31F008EF32F097
:1063D000000E58EC2AF061EC41F0000E58EC2AF067
:1063E00061EC47F001EC45F0000E58EC2AF031EC7E
:1063F00045F0000E58EC2AF061EC47F0FF0E58EC27
:106400002AF0F1EC41F0FF0E58EC2AF026EF32F0C2
:10641000FF0E58EC2AF001EC42F0FF0E58EC2AF087
:1064200061EC47F001EC45F0000E58EC2AF031EC3D
:1064300045F0000E58EC2AF061EC47F0000E58ECE5
:106440002AF051EC41F0000E58EC2AF04A50406E10
:106450003FA4120080BA35EF32F03EBA36EF32F088
:106460003F944A50406E3E8A12003E9A80B8AFEF89
:1064700032F03EB8B0EF32F0000E495CD8B461EFB4
:1064800032F0010E495CD8B46AEF32F0020E495C7A
:10649000D8B473EF32F0030E495CD8B47CEF32F01D
:1064A000040E495CD8B485EF32F0050E495CD8B4CF
:1064B0008EEF32F0060E495CD8B497EF32F0A0EFC1
:1064C00032F04BAE67EF32F04A8EA9EF32F04A9EBF
:1064D000A9EF32F04BAC70EF32F04A8CA9EF32F0FA
:1064E0004A9CA9EF32F04BAA79EF32F04A8AA9EF21
:1064F00032F04A9AA9EF32F04BA882EF32F04A8884
:10650000A9EF32F04A98A9EF32F04BA68BEF32F0A8
:106510004A86A9EF32F04A96A9EF32F04BA494EFE5
:1065200032F04A84A9EF32F04A94A9EF32F04BA23C
:106530009DEF32F04A82A9EF32F04A92A9EF32F091
:106540004BA0A6EF32F04A80A9EF32F04A90A9EFB3
:1065500032F03F944A50406E3E88B0EF32F03E98A1
:1065600080B0F4EF32F03EB0F5EF32F0000E495C4F
:10657000D8B4DBEF32F0010E495CD8B4DEEF32F074
:10658000020E495CD8B4E1EF32F0030E495CD8B496
:10659000E4EF32F0040E495CD8B4E7EF32F0050EB8
:1065A000495CD8B4EAEF32F0060E495CD8B4EDEF9E
:1065B00032F0F0EF32F04B7EF1EF32F04B7CF1EF46
:1065C00032F04B7AF1EF32F04B78F1EF32F04B765C
:1065D000F1EF32F04B74F1EF32F04B72F1EF32F039
:1065E0004B703E80F5EF32F03E9084B639EF33F0D9
:1065F0003EBC3AEF33F0000E495CD8B420EF33F0E4
:10660000010E495CD8B423EF33F0020E495CD8B4D4
:1066100026EF33F0030E495CD8B429EF33F0040EB3
:10662000495CD8B42CEF33F0050E495CD8B42FEF99
:1066300033F0060E495CD8B432EF33F035EF33F067
:106640004B7E36EF33F04B7C36EF33F04B7A36EF40
:1066500033F04B7836EF33F04B7636EF33F04B7444
:1066600036EF33F04B7236EF33F04B703E8C3AEF2F
:1066700033F03E9C120080B8ACEF33F03EB8ADEF83
:1066800033F0000E465CD8B474EF33F0010E465C74
:10669000D8B478EF33F0020E465CD8B47CEF33F018
:1066A000030E465CD8B480EF33F0040E465CD8B4D9
:1066B00084EF33F0050E465CD8B488EF33F0060E55
:1066C000465CD8B48CEF33F0070E465CD8B490EF3C
:1066D00033F0080E465CD8B494EF33F0090E465CF4
:1066E000D8B498EF33F012004A50116E9AEF33F09D
:1066F0004A50126E9AEF33F04A50136E9AEF33F00D
:106700004A50146E9AEF33F04A50156E9AEF33F0F8
:106710004A50166E9AEF33F04A50176E9AEF33F0E4
:106720004A50186E9AEF33F04A50196E9AEF33F0D0
:106730004A501A6E5FEC2BF04A50406E3E88000EB5
:10674000465CD8B4A8EF33F0070E496EADEF33F0D6
:10675000050E496EADEF33F03E9812001AEC2AF0A8
:10676000670E26EC2AF0BC0E3FEC2AF03FBCCDEFC2
:1067700033F0000E58EC2AF0A1EC45F0000E58EC76
:106780002AF071EC44F0000E58EC2AF041EC45F090
:10679000000E58EC2AF0DFEF33F0FF0E58EC2AF031
:1067A00041EC47F0FF0E58EC2AF001EC46F0FF0EEA
:1067B00058EC2AF0E1EC46F0FF0E58EC2AF01DEC04
:1067C0002AF0440E26EC2AF0BC0E3FEC2AF03FBC27
:1067D000FEEF33F0FF0E58EC2AF091EC46F0FF0E7E
:1067E00058EC2AF071EC47F0FF0E58EC2AF0A1ECBF
:1067F00046F0FF0E58EC2AF010EF34F0000E58EC83
:106800002AF0F1EC44F0000E58EC2AF061EC47F06D
:10681000000E58EC2AF001EC45F0000E58EC2AF07E
:1068200080B020EF34F03EB021EF34F03FBC1CEFDD
:1068300034F03F8C1DEF34F03F9C3E8021EF34F06C
:106840003E9084B631EF34F03EBC32EF34F03FBCC2
:106850002DEF34F03F8C2EEF34F03F9C3E8C32EF26
:1068600034F03E9C120080B8A7EF34F03EB8A8EF99
:1068700034F03FACA1EF34F042EC2BF0000E475C5B
:10688000D8B477EF34F0010E475CD8B47BEF34F026
:10689000020E475CD8B47FEF34F0030E475CD8B4E7
:1068A00083EF34F0040E475CD8B487EF34F0050E64
:1068B000475CD8B48BEF34F0060E475CD8B48FEF4A
:1068C00034F0070E475CD8B493EF34F0080E475C01
:1068D000D8B497EF34F0090E475CD8B49BEF34F08E
:1068E0000A0E475CD8B49FEF34F0A1EF34F099EC76
:1068F00047F0A1EF34F0ACEC47F0A1EF34F0BFEC7F
:1069000047F0A1EF34F0D2EC47F0A1EF34F0E5EC22
:1069100047F0A1EF34F0F8EC47F0A1EF34F00BECC6
:1069200048F0A1EF34F01EEC48F0A1EF34F031EC68
:1069300048F0A1EF34F044EC48F0A1EF34F057EC0C
:1069400048F0446A476A3F9C3E881BEF01F03E983E
:10695000120083A2C9EF34F03FB812004CB2BBEF73
:1069600034F01550380B406E180E406E1550C70BA2
:10697000156EC3EF34F015503F0B406E1B0E406E8A
:106980001550C00B156E405015125FEC2BF03F8870
:1069900012003F9812001550380B406E40424042A2
:1069A00040424050070B406E1550F80B156E40509A
:1069B00015121200106E000E105CD8A4F8EF34F01F
:1069C00005B8E9EF34F005BAEDEF34F0B1EC40F082
:1069D000120061EC47F0058C120005BCF4EF34F0B6
:1069E000059CB1EC40F01200059C61EC47F01200F0
:1069F000010E105CD8A400EF35F0C1EC40F012009D
:106A0000020E105CD8A408EF35F0D1EC40F0120073
:106A1000030E105CD8A410EF35F0E1EC40F012004A
:106A2000040E105CD8A418EF35F0F1EC40F0120021
:106A3000050E105CD8A420EF35F001EC41F01200F7
:106A4000060E105CD8A428EF35F011EC41F01200CE
:106A5000070E105CD8A430EF35F021EC41F01200A5
:106A6000080E105CD8A438EF35F031EC41F012007C
:106A700041EC41F01200106E000E105CD8A444EFFF
:106A800035F051EC41F01200010E105CD8A44CEF2F
:106A900035F061EC41F01200020E105CD8A454EF06
:106AA00035F071EC41F01200030E105CD8A45CEFDD
:106AB00035F081EC41F01200040E105CD8A464EFB4
:106AC00035F091EC41F01200050E105CD8A46CEF8B
:106AD00035F0A1EC41F01200060E105CD8A474EF62
:106AE00035F0B1EC41F01200070E105CD8A47CEF39
:106AF00035F0C1EC41F01200080E105CD8A484EF10
:106B000035F0D1EC41F01200E1EC41F01200106ED2
:106B1000000E105CD8A490EF35F0F1EC41F01200BB
:106B2000010E105CD8A498EF35F001EC42F0120091
:106B3000020E105CD8A4A0EF35F011EC42F0120068
:106B4000030E105CD8A4A8EF35F021EC42F012003F
:106B5000040E105CD8A4B0EF35F031EC42F0120016
:106B6000050E105CD8A4B8EF35F041EC42F01200ED
:106B7000060E105CD8A4C0EF35F051EC42F01200C4
:106B8000070E105CD8A4C8EF35F061EC42F012009B
:106B9000080E105CD8A4D0EF35F071EC42F0120072
:106BA00081EC42F01200062A0A0E065CD8A4D3EF4C
:106BB00035F0066A1200062AFF0E065CD8A4DBEF49
:106BC00035F0066A072A640E075CD8A4DBEF35F0BF
:106BD000066A076A1200062AFF0E065CD8A4EBEFCD
:106BE00035F0066A072AFF0E075CD8A4EBEF35F0F4
:106BF000066A076A12001AEC2AF0400E26EC2AF008
:106C0000BF0E3FEC2AF061EC44F0000E58EC2AF085
:106C100031EC44F0000E58EC2AF0B1EC44F0000ED8
:106C200058EC2AF0D1EC41F0000E58EC2AF091EC2F
:106C300041F0000E58EC2AF061EC41F0000E58ECE7
:106C40002AF0B1EC41F061EC47F031EC45F0000E78
:106C500058EC2AF071EC44F0000E58EC2AF071EC7C
:106C600045F01DEC2AF0400E26EC2AF0BF0E3FEC5A
:106C70002AF0400E58EC2AF0000E58EC2AF051ECA5
:106C800041F0000E58EC2AF0400E036E7F0E046EA9
:106C90001AEC2AF0035026EC2AF0BC0E3FEC2AF046
:106CA000010E58EC2AF01DEC2AF0045026EC2AF0D4
:106CB000BC0E3FEC2AF0010E58EC2AF0032A040621
:106CC000DBEC35F0800E035CD8A448EF36F0EBEC3B
:106CD00035F0EBEC35F0EBEC35F0EBEC35F0EBECC4
:106CE00035F0EBEC35F0400E036E7F0E046E1AECBF
:106CF0002AF0035026EC2AF0BC0E3FEC2AF0000EDE
:106D000058EC2AF01DEC2AF0045026EC2AF0BC0EB8
:106D10003FEC2AF0000E58EC2AF0032A0406DBECC4
:106D200035F0800E035CD8A477EF36F03F8EEBECA5
:106D300035F0EBEC35F0EBEC35F0EBEC35F0EBEC63
:106D400035F050801AEC2AF04A0E26EC2AF0BB0EE1
:106D50003FEC2AF0E1EC42F0000E58EC2AF0100E65
:106D600058EC2AF0100E58EC2AF0100E58EC2AF0CD
:106D7000100E58EC2AF0100E58EC2AF0000E58ECC9
:106D80002AF061EC43F0000E58EC2AF061EC47F079
:106D9000000E58EC2AF0D1EC42F0000E58EC2AF02C
:106DA00061EC43F0000E58EC2AF0F1EC42F0000EDA
:106DB00058EC2AF011EC43F0000E58EC2AF061EC8C
:106DC00043F0000E58EC2AF01DEC2AF0400E26ECA1
:106DD0002AF0BB0E3FEC2AF0D1EC42F0000E58EC4A
:106DE0002AF0D1EC42F0000E58EC2AF0A1EC43F06E
:106DF000000E58EC2AF011EC43F0000E58EC2AF08B
:106E000061EC43F0000E58EC2AF0F1EC42F0000E79
:106E100058EC2AF050901AEC2AF0560E26EC2AF084
:106E2000BC0E3FEC2AF091EC42F0000E58EC2AF038
:106E3000D1EC43F0000E58EC2AF0C1EC42F0000E09
:106E400058EC2AF011EC43F0000E58EC2AF071ECEB
:106E500043F0000E58EC2AF061EC47F0000E58ECBD
:106E60002AF041EC43F0000E58EC2AF01DEC2AF019
:106E7000400E26EC2AF0BC0E3FEC2AF091EC42F0DA
:106E8000000E58EC2AF0A1EC42F0000E58EC2AF06B
:106E900071EC43F0000E58EC2AF0A1EC43F0000E28
:106EA00058EC2AF091EC42F0000E58EC2AF0C1ECBC
:106EB00043F0000E58EC2AF071EC43F0000E58EC51
:106EC0002AF0A1EC43F0000E58EC2AF011EC44F04B
:106ED000000E58EC2AF0512A080E515CD8A497EF06
:106EE00036F03F9E516AEBEC35F0EBEC35F0EBEC15
:106EF00035F0EBEC35F0EBEC35F0EBEC35F0EBECA2
:106F000035F0EBEC35F0EBEC35F0EBEC35F0EBEC91
:106F100035F0EBEC35F0EBEC35F0EBEC35F0EBEC81
:106F200035F0EBEC35F0EBEC35F0EBEC35F0EBEC71
:106F300035F0EBEC35F0EBEC35F0EBEC35F0EBEC61
:106F400035F0EBEC35F0EBEC35F0EBEC35F0EBEC51
:106F500035F0EBEC35F0EBEC35F0EBEC35F0EBEC41
:106F600035F0EBEC35F0EBEC35F0EBEC35F0EBEC31
:106F700035F0EBEC35F0EBEC35F0EBEC35F0EBEC21
:106F800035F0EBEC35F0EBEC35F0EBEC35F0EBEC11
:106F900035F0EBEC35F0EBEC35F0EBEC35F0EBEC01
:106FA00035F0EBEC35F0EBEC35F0EBEC35F0EBECF1
:106FB00035F0EBEC35F0EBEC35F0EBEC35F0EBECE1
:106FC00035F0EBEC35F0EBEC35F0EBEC35F0EBECD1
:106FD00035F0EBEC35F0EBEC35F0EBEC35F0EBECC1
:106FE00035F0EBEC35F0EBEC35F0EBEC35F0EBECB1
:106FF00035F0EBEC35F0EBEC35F0EBEC35F0EBECA1
:1070000035F0EBEC35F0EBEC35F0EBEC35F0EBEC90
:1070100035F0EBEC35F0EBEC35F0EBEC35F0EBEC80
:1070200035F0EBEC35F0EBEC35F0EBEC35F0EBEC70
:1070300035F0EBEC35F0EBEC35F0EBEC35F0EBEC60
:1070400035F0EBEC35F0EBEC35F0EBEC35F0EBEC50
:1070500035F0EBEC35F0EBEC35F0EBEC35F0EBEC40
:1070600035F0EBEC35F0EBEC35F0EBEC35F0EBEC30
:1070700035F0EBEC35F0EBEC35F0EBEC35F0EBEC20
:1070800035F0EBEC35F0EBEC35F0EBEC35F042ECB9
:107090002BF0EBEC35F0EBEC35F0EBEC35F0EBEC0A
:1070A00035F0EBEC35F0EBEC35F0EBEC35F01200B5
:1070B000096E640E095ED8A061EF38F00A2A59EF14
:1070C00038F0640E09260A0E095ED8A06BEF38F07E
:1070D0000B2A63EF38F00A0E0926010E095ED8A0CC
:1070E00075EF38F00C2A6DEF38F012000D6E100EAF
:1070F0000D5ED8A07FEF38F00B2A77EF38F0100E36
:107100000D26010E0D5ED8A089EF38F00C2A81EF14
:1071100038F0120005880A50DAEC34F0000E58EC12
:107120002AF00598058A0B50DAEC34F0000E58EC82
:107130002AF0059A0C50DAEC34F0000E58EC2AF0E4
:107140000A6A0B6A0C6A12000A503BEC35F0000E1A
:1071500058EC2AF00B503BEC35F0000E58EC2AF0BE
:107160000C503BEC35F0000E58EC2AF00A6A0B6A22
:107170000C6A12000A5087EC35F0FF0E58EC2AF02A
:107180000B5087EC35F0FF0E58EC2AF00C5087ECD2
:1071900035F0FF0E58EC2AF00A6A0B6A0C6A1200EE
:1071A000406E452A090E455CD8B4E6EF38F040BE83
:1071B000DEEF38F051EC41F0E0EF38F061EC41F0F7
:1071C000000E58EC2AF04046D1EF38F0456A120024
:1071D000406E080E455CD8B425EF39F040BE0AEF8A
:1071E00039F04550495CD8B400EF39F0000E58EC46
:1071F0002AF051EC41F0000E58EC2AF021EF39F062
:10720000FF0E58EC2AF0F1EC41F0FF0E58EC2AF09A
:1072100021EF39F04550495CD8B419EF39F0000E30
:1072200058EC2AF061EC41F0000E58EC2AF021EF06
:1072300039F0FF0E58EC2AF001EC42F0FF0E58EC4A
:107240002AF0452A4046E9EF38F0456A1200C80E98
:107250004F5CD8B42EEF39F04F2A12003F8A4F6AA4
:1072600012001DEC2AF0530E26EC2AF0BE0E3FEC65
:107270002AF0080E495CD8A489EF39F0FF0E58ECCB
:107280002AF0E1EC46F0FF0E58EC2AF001EC46F053
:10729000FF0E58EC2AF0F1EC46F0FF0E58EC2AF005
:1072A0001AEC2AF0460E26EC2AF0BC0E3FEC2AF02F
:1072B000000E58EC2AF061EC47F0000E58EC2AF072
:1072C00061EC47F0000E58EC2AF061EC47F0000E3C
:1072D00058EC2AF061EC47F0000E58EC2AF061EC13
:1072E00047F0000E58EC2AF061EC47F0000E58EC25
:1072F0002AF061EC47F0000E58EC2AF061EC47F000
:10730000000E58EC2AF061EC47F0000E58EC2AF021
:107310001200000E58EC2AF041EC45F0000E58EC3B
:107320002AF071EC44F0000E58EC2AF051EC45F0D4
:10733000000E58EC2AF012001DEC2AF0400E26EC4C
:107340002AF0BB0E3FEC2AF01200000E58EC2AF097
:10735000F1EC44F0000E58EC2AF001EC45F0000E80
:1073600058EC2AF061EC47F0000E58EC2AF027ECBC
:107370003BF061EC47F0000E58EC2AF061EC47F06E
:1073800061EC47F082EC3BF01200FF0E58EC2AF063
:10739000C1EC46F0FF0E58EC2AF0E1EC45F0FF0E90
:1073A00058EC2AF0D1EC46F0FF0E58EC2AF0E1EC54
:1073B00045F0FF0E58EC2AF071EC47F0FF0E58EC48
:1073C0002AF041EC3BF082EC3BF01200FF0E58EC4F
:1073D0002AF0E1EC45F0FF0E58EC2AF0E1EC45F024
:1073E000FF0E58EC2AF0D1EC46F0FF0E58EC2AF0D4
:1073F000E1EC45F0FF0E58EC2AF071EC47F0FF0E7F
:1074000058EC2AF041EC3BF082EC3BF01200FF0E0E
:1074100058EC2AF001EC47F0FF0E58EC2AF091EC02
:1074200046F0FF0E58EC2AF071EC46F0FF0E58ECD7
:107430002AF0A1EC46F0FF0E58EC2AF0E1EC45F002
:10744000FF0E58EC2AF061EC46F0FF0E58EC2AF0E3
:1074500061EC47F0000E58EC2AF061EC47F0000EAA
:1074600058EC2AF061EC47F0000E58EC2AF061EC81
:1074700047F0000E58EC2AF082EC3BF01200FF0EB1
:1074800058EC2AF011EC47F0FF0E58EC2AF0C1EC52
:1074900045F0FF0E58EC2AF071EC46F0FF0E58EC68
:1074A0002AF041EC46F0FF0E58EC2AF0F1EC45F0E2
:1074B000FF0E58EC2AF041EC46F0FF0E58EC2AF093
:1074C000F1EC46F0FF0E58EC2AF041EC47F0FF0ECD
:1074D00058EC2AF071EC47F001EC46F0FF0E58EC46
:1074E0002AF0810E58EC2AF0ED0E58EC2AF0ED0E41
:1074F00058EC2AF0ED0E58EC2AF09CEC39F0930E83
:1075000058EC2AF0FF0E58EC2AF04BEC3BF061EC03
:1075100047F0000E58EC2AF01200FF0E58EC2AF04B
:10752000D1EC45F0FF0E58EC2AF041EC46F0FF0E8E
:1075300058EC2AF071EC47F0FF0E58EC2AF0B1EC51
:1075400046F0FF0E58EC2AF031EC46F0FF0E58ECF6
:107550002AF0C1EC45F0FF0E58EC2AF0E1EC46F0C1
:10756000FF0E58EC2AF001EC46F0FF0E58EC2AF022
:1075700071EC47F001EC46F0FF0E58EC2AF0810E5A
:1075800058EC2AF0ED0E58EC2AF0ED0E58EC2AF0EB
:10759000ED0E58EC2AF09CEC39F0930E58EC2AF0E2
:1075A000FF0E58EC2AF04BEC3BF061EC47F0000E7C
:1075B00058EC2AF01200FF0E58EC2AF0B1EC46F01D
:1075C000FF0E58EC2AF0C1EC45F0FF0E58EC2AF003
:1075D000D1EC46F0FF0E58EC2AF041EC46F0FF0EDD
:1075E00058EC2AF0F1EC46F0FF0E58EC2AF041EC92
:1075F00047F0FF0E58EC2AF071EC47F001EC46F032
:10760000FF0E58EC2AF0D1EC46F0FF0E58EC2AF0B1
:10761000D1EC46F0FF0E58EC2AF0C30E58EC2AF0DD
:10762000BD0E58EC2AF0BD0E58EC2AF0BD0E58ECF9
:107630002AF09CEC39F0C30E58EC2AF0FF0E58ECFF
:107640002AF055EC3BF0000E58EC2AF0120071ECD9
:1076500044F0000E58EC2AF031EC45F0000E58ECE6
:107660002AF031EC45F0000E58EC2AF001EC45F020
:10767000000E58EC2AF031EC45F0000E58EC2AF0E0
:10768000120001EC46F0FF0E58EC2AF0D1EC46F067
:10769000FF0E58EC2AF0D1EC46F0FF0E58EC2AF021
:1076A000A1EC46F0FF0E58EC2AF0D1EC46F0FF0EAC
:1076B00058EC2AF0120041EC3BF071EC47F0FF0E61
:1076C00058EC2AF0E1EC45F0FF0E58EC2AF0A1EC62
:1076D00046F0FF0E58EC2AF0F1EC45F0FF0E58ECA6
:1076E0002AF001EC46F0FF0E58EC2AF0FF0E58ECA1
:1076F0002AF0FF0E58EC2AF0FF0E58EC2AF09CEC12
:1077000039F012009CEC39F061EC47F0000E58ECB7
:107710002AF061EC47F0000E58EC2AF061EC47F0DB
:10772000000E58EC2AF061EC47F0000E58EC2AF0FD
:1077300061EC47F0000E58EC2AF0120051EC44F0D6
:10774000000E58EC2AF001EC45F0000E58EC2AF03F
:10775000F1EC44F0000E58EC2AF051EC45F0000E2C
:1077600058EC2AF031EC45F0000E58EC2AF001EC10
:1077700045F0000E58EC2AF0D1EC44F0000E58EC25
:107780002AF061EC47F051EC41F0000E58EC2AF081
:1077900061EC47F01DEC2AF0400E26EC2AF0B90E01
:1077A0003FEC2AF0FF0E58EC2AF0810E58EC2AF03C
:1077B000810E58EC2AF0000E58EC2AF051EC41F002
:1077C000000E58EC2AF051EC41F0000E58EC2AF073
:1077D000A1EC44F0000E58EC2AF0810E58EC2AF08F
:1077E000810E58EC2AF0FF0E58EC2AF0120051ECF2
:1077F00044F0000E58EC2AF001EC45F0000E58EC75
:107800002AF0F1EC44F0000E58EC2AF051EC45F06F
:10781000000E58EC2AF031EC45F0000E58EC2AF03E
:1078200001EC45F0000E58EC2AF0D1EC44F0000ECB
:1078300058EC2AF061EC47F061EC41F0000E58EC96
:107840002AF061EC47F01DEC2AF0400E26EC2AF0FD
:10785000B90E3FEC2AF0FF0E58EC2AF0810E58ECDE
:107860002AF0810E58EC2AF0000E58EC2AF051EC68
:1078700041F0000E58EC2AF061EC41F0000E58EC9B
:107880002AF0A1EC44F0000E58EC2AF0810E58ECDE
:107890002AF0810E58EC2AF0FF0E58EC2AF0120064
:1078A00051EC44F0000E58EC2AF001EC45F0000ECB
:1078B00058EC2AF0F1EC44F0000E58EC2AF051ECB0
:1078C00045F0000E58EC2AF031EC45F0000E58EC73
:1078D0002AF001EC45F0000E58EC2AF0D1EC44F00F
:1078E000000E58EC2AF061EC47F071EC41F0000E0C
:1078F00058EC2AF061EC47F01DEC2AF0400E26EC23
:107900002AF0B90E3FEC2AF0FF0E58EC2AF0810E57
:1079100058EC2AF0810E58EC2AF0000E58EC2AF0B0
:1079200051EC41F0000E58EC2AF071EC41F0000EE1
:1079300058EC2AF0A1EC44F0000E58EC2AF0810E2D
:1079400058EC2AF0810E58EC2AF0FF0E58EC2AF081
:10795000120051EC44F0000E58EC2AF001EC45F016
:10796000000E58EC2AF0F1EC44F0000E58EC2AF02E
:1079700051EC45F0000E58EC2AF031EC45F0000EC9
:1079800058EC2AF001EC45F0000E58EC2AF0D1EC4E
:1079900044F0000E58EC2AF061EC47F081EC41F025
:1079A000000E58EC2AF061EC47F01DEC2AF0400E76
:1079B00026EC2AF0B90E3FEC2AF0FF0E58EC2AF024
:1079C000810E58EC2AF0810E58EC2AF0000E58EC8B
:1079D0002AF051EC41F0000E58EC2AF081EC41F015
:1079E000000E58EC2AF0A1EC44F0000E58EC2AF0FE
:1079F000810E58EC2AF0810E58EC2AF0FF0E58EC5C
:107A00002AF0120051EC44F0000E58EC2AF001EC80
:107A100045F0000E58EC2AF0F1EC44F0000E58EC62
:107A20002AF051EC45F0000E58EC2AF031EC45F00C
:107A3000000E58EC2AF001EC45F0000E58EC2AF04C
:107A4000D1EC44F0000E58EC2AF061EC47F091ECD8
:107A500041F0000E58EC2AF061EC47F01DEC2AF0E2
:107A6000400E26EC2AF0B90E3FEC2AF0FF0E58EC3F
:107A70002AF0810E58EC2AF0810E58EC2AF0000E04
:107A800058EC2AF051EC41F0000E58EC2AF091EC41
:107A900041F0000E58EC2AF0A1EC44F0000E58EC36
:107AA0002AF0810E58EC2AF0810E58EC2AF0FF0ED5
:107AB00058EC2AF0120041EC45F0000E58EC2AF088
:107AC00071EC44F0000E58EC2AF031EC45F0000E59
:107AD00058EC2AF0B1EC44F0000E58EC2AF031ECEE
:107AE00044F0000E58EC2AF0D1EC44F0000E58ECB3
:107AF0002AF061EC47F031EC44F0000E58EC2AF02B
:107B000061EC45F0000E58EC2AF061EC44F01DECFD
:107B10002AF0400E26EC2AF0B90E3FEC2AF0000EB7
:107B200058EC2AF0B1EC44F0000E58EC2AF001ECCD
:107B300045F0000E58EC2AF01AEC2AF04C0E26EC18
:107B40002AF0BA0E3FEC2AF061EC44F0000E58EC3B
:107B50002AF031EC44F0000E58EC2AF051EC45F0DC
:107B6000000E58EC2AF031EC44F0000E58EC2AF0EC
:107B700061EC47F081EC44F0000E58EC2AF001EC87
:107B800045F0000E58EC2AF031EC45F0000E58ECB0
:107B90002AF0E1EC44F01DEC2AF0400E26EC2AF02D
:107BA000BA0E3FEC2AF0000E58EC2AF031EC44F00B
:107BB000000E58EC2AF051EC45F061EC47F0FF0E56
:107BC00058EC2AF0810E58EC2AF0810E58EC2AF07D
:107BD000000E58EC2AF051EC41F0000E58EC2AF05F
:107BE000A1EC41F0000E58EC2AF0A1EC44F0000E9C
:107BF00058EC2AF0810E58EC2AF0810E58EC2AF04D
:107C0000FF0E58EC2AF0120031EC45F0000E58EC53
:107C10002AF071EC44F0000E58EC2AF051EC44F0DC
:107C2000000E58EC2AF071EC44F0000E58EC2AF0EB
:107C3000B1EC44F0000E58EC2AF071EC45F0000E67
:107C400058EC2AF071EC44F0000E58EC2AF031ECBC
:107C500045F0000E58EC2AF061EC47F071EC44F06E
:107C60001DEC2AF0400E26EC2AF0B90E3FEC2AF06B
:107C7000000E58EC2AF031EC45F0000E58EC2AF0DA
:107C800031EC45F0000E58EC2AF001EC45F0000E06
:107C900058EC2AF031EC45F0000E58EC2AF061EC7B
:107CA00047F0E1EC44F0000E58EC2AF031EC44F0DF
:107CB000000E58EC2AF041EC45F0000E58EC2AF08A
:107CC000C1EC44F0000E58EC2AF01DEC2AF0640ED2
:107CD00026EC2AF0BA0E3FEC2AF0FF0E58EC2AF000
:107CE000810E58EC2AF0810E58EC2AF0000E58EC68
:107CF0002AF051EC41F0000E58EC2AF0B1EC41F0C2
:107D0000000E58EC2AF0A1EC44F0000E58EC2AF0DA
:107D1000810E58EC2AF0810E58EC2AF0FF0E58EC38
:107D20002AF01200B1EC44F0000E58EC2AF0F1EC0D
:107D300044F0000E58EC2AF051EC45F0000E58ECDF
:107D40002AF071EC44F0000E58EC2AF031EC45F0CA
:107D5000000E58EC2AF031EC45F0000E58EC2AF0F9
:107D600061EC45F0000E58EC2AF011EC45F0000EE5
:107D700058EC2AF051EC45F061EC47F01DEC2AF08C
:107D8000400E26EC2AF0B90E3FEC2AF0000E58EC1B
:107D90002AF0E1EC44F0000E58EC2AF031EC44F00B
:107DA000000E58EC2AF041EC45F0000E58EC2AF099
:107DB000C1EC44F061EC47F0FF0E58EC2AF0810E64
:107DC00058EC2AF0810E58EC2AF0000E58EC2AF0FC
:107DD00051EC41F0000E58EC2AF0C1EC41F0000EDD
:107DE00058EC2AF0A1EC44F0000E58EC2AF0810E79
:107DF00058EC2AF0810E58EC2AF0FF0E58EC2AF0CD
:107E00001200B1EC44F0000E58EC2AF0F1EC44F012
:107E1000000E58EC2AF051EC45F0000E58EC2AF018
:107E200071EC44F0000E58EC2AF031EC45F0000EF5
:107E300058EC2AF031EC45F0000E58EC2AF061ECD9
:107E400045F0000E58EC2AF011EC45F0000E58EC0D
:107E50002AF051EC45F061EC47F01DEC2AF0400EA1
:107E600026EC2AF0B90E3FEC2AF0000E58EC2AF06E
:107E7000E1EC44F0000E58EC2AF001EC45F0000E65
:107E800058EC2AF061EC44F0000E58EC2AF071EC4A
:107E900044F0000E58EC2AF061EC47F0E1EC44F0BD
:107EA000000E58EC2AF041EC45F0000E58EC2AF098
:107EB00041EC44F0000E58EC2AF01DEC2AF0640E60
:107EC00026EC2AF0BA0E3FEC2AF0FF0E58EC2AF00E
:107ED000810E58EC2AF0810E58EC2AF0000E58EC76
:107EE0002AF051EC41F0000E58EC2AF0D1EC41F0B0
:107EF000000E58EC2AF0A1EC44F0000E58EC2AF0E9
:107F0000810E58EC2AF0810E58EC2AF0FF0E58EC46
:107F10002AF01200B1EC44F0000E58EC2AF0F1EC1B
:107F200044F0000E58EC2AF051EC45F0000E58ECED
:107F30002AF071EC44F0000E58EC2AF031EC45F0D8
:107F4000000E58EC2AF031EC45F0000E58EC2AF007
:107F500061EC45F0000E58EC2AF011EC45F0000EF3
:107F600058EC2AF051EC45F061EC47F01DEC2AF09A
:107F7000400E26EC2AF0B90E3FEC2AF0000E58EC29
:107F80002AF0E1EC44F0000E58EC2AF001EC45F048
:107F9000000E58EC2AF061EC44F0000E58EC2AF088
:107FA00071EC44F0000E58EC2AF061EC47F0D1EC93
:107FB00044F0000E58EC2AF041EC45F0000E58EC6D
:107FC0002AF041EC44F0000E58EC2AF01DEC2AF0A7
:107FD000640E26EC2AF0BA0E3FEC2AF0FF0E58ECA5
:107FE0002AF0810E58EC2AF0810E58EC2AF0000E8F
:107FF00058EC2AF051EC41F0000E58EC2AF0E1EC7C
:1080000041F0000E58EC2AF0A1EC44F0000E58ECC0
:108010002AF0810E58EC2AF0810E58EC2AF0FF0E5F
:1080200058EC2AF01200FF0E58EC2AF0B1EC46F0A2
:10803000FF0E58EC2AF0E1EC45F0FF0E58EC2AF068
:10804000E1EC45F0FF0E58EC2AF031EC46F0FF0E63
:1080500058EC2AF01200FF0E58EC2AF0A1EC46F082
:10806000FF0E58EC2AF0E1EC46F0FF0E58EC2AF037
:1080700071EC46F0FF0E58EC2AF041EC46F0FF0E92
:1080800058EC2AF0B1EC46F0FF0E58EC2AF0120042
:10809000FF0E58EC2AF0F1EC45F0FF0E58EC2AF0F8
:1080A00001EC46F0FF0E58EC2AF0F1EC46F0FF0E22
:1080B00058EC2AF0E1EC45F0FF0E58EC2AF01200E3
:1080C000FF0E58EC2AF0E1EC45F0FF0E58EC2AF0D8
:1080D000E1EC45F0FF0E58EC2AF031EC46F0FF0ED3
:1080E00058EC2AF01200FF0E58EC2AF0D1EC46F0C2
:1080F000FF0E58EC2AF001EC46F0FF0E58EC2AF087
:10810000D1EC46F0FF0E58EC2AF0D1EC46F0FF0E11
:1081100058EC2AF01200FF0E58EC2AF0C1EC46F0A1
:10812000FF0E58EC2AF0E1EC45F0FF0E58EC2AF077
:1081300031EC46F0FF0E58EC2AF01200FF0E58EC1E
:108140002AF011EC46F0FF0E58EC2AF0E1EC45F075
:10815000FF0E58EC2AF031EC46F0FF0E58EC2AF0F6
:1081600012007C0E58EC2AF0820E58EC2AF0820E97
:1081700058EC2AF0820E58EC2AF07C0E58EC2AF0CB
:108180001200000E58EC2AF0840E58EC2AF0FE0E75
:1081900058EC2AF0800E58EC2AF0000E58EC2AF029
:1081A0001200E20E58EC2AF0920E58EC2AF0920ED1
:1081B00058EC2AF0920E58EC2AF08C0E58EC2AF06B
:1081C0001200440E58EC2AF0820E58EC2AF0920E5F
:1081D00058EC2AF0920E58EC2AF06C0E58EC2AF06B
:1081E0001200300E58EC2AF0280E58EC2AF0240E1B
:1081F00058EC2AF0FE0E58EC2AF0200E58EC2AF02B
:1082000012004E0E58EC2AF08A0E58EC2AF08A0E14
:1082100058EC2AF08A0E58EC2AF0720E58EC2AF02C
:1082200012007C0E58EC2AF0920E58EC2AF0920EB6
:1082300058EC2AF0920E58EC2AF0640E58EC2AF012
:108240001200060E58EC2AF0020E58EC2AF0C20E6C
:1082500058EC2AF0320E58EC2AF00E0E58EC2AF0A8
:1082600012006C0E58EC2AF0920E58EC2AF0920E86
:1082700058EC2AF0920E58EC2AF06C0E58EC2AF0CA
:1082800012004C0E58EC2AF0920E58EC2AF0920E86
:1082900058EC2AF0920E58EC2AF07C0E58EC2AF09A
:1082A00012003C0E58EC2AF0420E58EC2AF0420E16
:1082B00058EC2AF0420E58EC2AF03C0E58EC2AF00A
:1082C0001200000E58EC2AF0440E58EC2AF07E0EF4
:1082D00058EC2AF0400E58EC2AF0000E58EC2AF028
:1082E0001200720E58EC2AF04A0E58EC2AF04A0E90
:1082F00058EC2AF04A0E58EC2AF0440E58EC2AF0BA
:108300001200220E58EC2AF04A0E58EC2AF04A0EBF
:1083100058EC2AF04A0E58EC2AF0340E58EC2AF0A9
:108320001200300E58EC2AF0280E58EC2AF0240ED9
:1083300058EC2AF07E0E58EC2AF0200E58EC2AF069
:1083400012002E0E58EC2AF04A0E58EC2AF04A0E73
:1083500058EC2AF04A0E58EC2AF0320E58EC2AF06B
:1083600012003C0E58EC2AF04A0E58EC2AF04A0E45
:1083700058EC2AF04A0E58EC2AF0300E58EC2AF04D
:108380001200060E58EC2AF0020E58EC2AF0620E8B
:1083900058EC2AF0120E58EC2AF00E0E58EC2AF087
:1083A0001200340E58EC2AF04A0E58EC2AF04A0E0D
:1083B00058EC2AF04A0E58EC2AF0340E58EC2AF009
:1083C00012000C0E58EC2AF0520E58EC2AF0520E05
:1083D00058EC2AF0520E58EC2AF03C0E58EC2AF0D9
:1083E0001200C30E58EC2AF0BD0E58EC2AF0BD0E58
:1083F00058EC2AF0BD0E58EC2AF0C30E58EC2AF0C7
:108400001200FF0E58EC2AF0BB0E58EC2AF0810E39
:1084100058EC2AF0BF0E58EC2AF0FF0E58EC2AF068
:1084200012008D0E58EC2AF0B50E58EC2AF0B50E5D
:1084300058EC2AF0B50E58EC2AF0BB0E58EC2AF096
:108440001200DD0E58EC2AF0B50E58EC2AF0B50EED
:1084500058EC2AF0B50E58EC2AF0CB0E58EC2AF066
:108460001200CF0E58EC2AF0D70E58EC2AF0DB0E93
:1084700058EC2AF0810E58EC2AF0DF0E58EC2AF066
:108480001200D10E58EC2AF0B50E58EC2AF0B50EB9
:1084900058EC2AF0B50E58EC2AF0CD0E58EC2AF024
:1084A0001200C30E58EC2AF0B50E58EC2AF0B50EA7
:1084B00058EC2AF0B50E58EC2AF0CF0E58EC2AF002
:1084C0001200F90E58EC2AF0FD0E58EC2AF09D0E21
:1084D00058EC2AF0ED0E58EC2AF0F10E58EC2AF088
:1084E0001200CB0E58EC2AF0B50E58EC2AF0B50E5F
:1084F00058EC2AF0B50E58EC2AF0CB0E58EC2AF0C6
:108500001200F30E58EC2AF0AD0E58EC2AF0AD0E26
:1085100058EC2AF0AD0E58EC2AF0C30E58EC2AF0B5
:108520001200F80E58EC2AF0240E58EC2AF0220E15
:1085300058EC2AF0240E58EC2AF0F80E58EC2AF0E9
:108540001200FE0E58EC2AF0920E58EC2AF0920E11
:1085500058EC2AF0920E58EC2AF06C0E58EC2AF0E7
:1085600012007C0E58EC2AF0820E58EC2AF0820E93
:1085700058EC2AF0820E58EC2AF0440E58EC2AF0FF
:108580001200FE0E58EC2AF0820E58EC2AF0820EF1
:1085900058EC2AF0820E58EC2AF07C0E58EC2AF0A7
:1085A0001200FE0E58EC2AF0920E58EC2AF0920EB1
:1085B00058EC2AF0920E58EC2AF0820E58EC2AF071
:1085C0001200FE0E58EC2AF0120E58EC2AF0120E91
:1085D00058EC2AF0120E58EC2AF0020E58EC2AF051
:1085E00012007C0E58EC2AF0820E58EC2AF0820E13
:1085F00058EC2AF0920E58EC2AF0740E58EC2AF03F
:108600001200FE0E58EC2AF0100E58EC2AF0100E54
:1086100058EC2AF0100E58EC2AF0FE0E58EC2AF016
:108620001200000E58EC2AF0820E58EC2AF0FE0ED2
:1086300058EC2AF0820E58EC2AF0000E58EC2AF082
:108640001200600E58EC2AF0800E58EC2AF0800ED2
:1086500058EC2AF0800E58EC2AF07E0E58EC2AF0E6
:108660001200FE0E58EC2AF0100E58EC2AF0280EDC
:1086700058EC2AF0440E58EC2AF0820E58EC2AF0FE
:108680001200FE0E58EC2AF0800E58EC2AF0800EF4
:1086900058EC2AF0800E58EC2AF0800E58EC2AF0A4
:1086A0001200FE0E58EC2AF0040E58EC2AF0080EC8
:1086B00058EC2AF0040E58EC2AF0FE0E58EC2AF082
:1086C0001200FE0E58EC2AF0080E58EC2AF0100E9C
:1086D00058EC2AF0200E58EC2AF0FE0E58EC2AF046
:1086E00012007C0E58EC2AF0820E58EC2AF0820E12
:1086F00058EC2AF0820E58EC2AF07C0E58EC2AF046
:108700001200FE0E58EC2AF0120E58EC2AF0120E4F
:1087100058EC2AF0120E58EC2AF00C0E58EC2AF005
:1087200012007C0E58EC2AF0820E58EC2AF0A20EB1
:1087300058EC2AF0420E58EC2AF0BC0E58EC2AF005
:108740001200FE0E58EC2AF0120E58EC2AF0120E0F
:1087500058EC2AF0120E58EC2AF0EC0E58EC2AF0E5
:1087600012004C0E58EC2AF0920E58EC2AF0920EA1
:1087700058EC2AF0920E58EC2AF0640E58EC2AF0CD
:108780001200020E58EC2AF0020E58EC2AF0FE0EEF
:1087900058EC2AF0020E58EC2AF0020E58EC2AF09F
:1087A00012007E0E58EC2AF0800E58EC2AF0800E53
:1087B00058EC2AF0800E58EC2AF07E0E58EC2AF085
:1087C00012000E0E58EC2AF0300E58EC2AF0C00EB3
:1087D00058EC2AF0300E58EC2AF00E0E58EC2AF025
:1087E00012001E0E58EC2AF0E00E58EC2AF0180E7B
:1087F00058EC2AF0E00E58EC2AF01E0E58EC2AF045
:108800001200C60E58EC2AF0280E58EC2AF0100E72
:1088100058EC2AF0280E58EC2AF0C60E58EC2AF034
:1088200012000E0E58EC2AF0100E58EC2AF0E00E52
:1088300058EC2AF0100E58EC2AF00E0E58EC2AF0E4
:108840001200C20E58EC2AF0A20E58EC2AF0920E3A
:1088500058EC2AF08A0E58EC2AF0860E58EC2AF0D2
:108860001200780E58EC2AF0140E58EC2AF0120E72
:1088700058EC2AF0140E58EC2AF0780E58EC2AF036
:1088800012007E0E58EC2AF04A0E58EC2AF04A0EDE
:1088900058EC2AF04A0E58EC2AF0340E58EC2AF024
:1088A00012003C0E58EC2AF0420E58EC2AF0420E10
:1088B00058EC2AF0420E58EC2AF0240E58EC2AF01C
:1088C00012007E0E58EC2AF0420E58EC2AF0420EAE
:1088D00058EC2AF0420E58EC2AF03C0E58EC2AF0E4
:1088E00012007E0E58EC2AF04A0E58EC2AF04A0E7E
:1088F00058EC2AF04A0E58EC2AF0420E58EC2AF0B6
:1089000012007E0E58EC2AF00A0E58EC2AF00A0EDD
:1089100058EC2AF00A0E58EC2AF0020E58EC2AF015
:1089200012003C0E58EC2AF0420E58EC2AF0420E8F
:1089300058EC2AF0520E58EC2AF0340E58EC2AF07B
:1089400012007E0E58EC2AF0080E58EC2AF0080EA1
:1089500058EC2AF0080E58EC2AF07E0E58EC2AF05B
:108960001200000E58EC2AF0420E58EC2AF07E0E4F
:1089700058EC2AF0420E58EC2AF0000E58EC2AF07F
:1089800012007E0E58EC2AF0100E58EC2AF0080E59
:1089900058EC2AF0140E58EC2AF0620E58EC2AF02B
:1089A00012007E0E58EC2AF0400E58EC2AF0400ED1
:1089B00058EC2AF0400E58EC2AF0400E58EC2AF001
:1089C00012007E0E58EC2AF0040E58EC2AF0080E25
:1089D00058EC2AF0040E58EC2AF07E0E58EC2AF0DF
:1089E00012007E0E58EC2AF0040E58EC2AF0180EF5
:1089F00058EC2AF0200E58EC2AF07E0E58EC2AF0A3
:108A000012003C0E58EC2AF0420E58EC2AF0420EAE
:108A100058EC2AF0420E58EC2AF03C0E58EC2AF0A2
:108A200012007E0E58EC2AF0120E58EC2AF0120EAC
:108A300058EC2AF0120E58EC2AF00C0E58EC2AF0E2
:108A400012003C0E58EC2AF0420E58EC2AF0520E5E
:108A500058EC2AF0220E58EC2AF05C0E58EC2AF062
:108A600012007E0E58EC2AF0120E58EC2AF0120E6C
:108A700058EC2AF0120E58EC2AF06C0E58EC2AF042
:108A80001200440E58EC2AF04A0E58EC2AF04A0E16
:108A900058EC2AF04A0E58EC2AF0320E58EC2AF024
:108AA0001200020E58EC2AF0020E58EC2AF07E0E4C
:108AB00058EC2AF0020E58EC2AF0020E58EC2AF07C
:108AC00012003E0E58EC2AF0400E58EC2AF0400EF0
:108AD00058EC2AF0400E58EC2AF03E0E58EC2AF0E2
:108AE0001200060E58EC2AF0180E58EC2AF0600E10
:108AF00058EC2AF0180E58EC2AF0060E58EC2AF022
:108B000012007E0E58EC2AF0200E58EC2AF0100EBF
:108B100058EC2AF0200E58EC2AF07E0E58EC2AF081
:108B20001200460E58EC2AF0280E58EC2AF0100ECF
:108B300058EC2AF0280E58EC2AF0460E58EC2AF091
:108B40001200060E58EC2AF0080E58EC2AF0700EAF
:108B500058EC2AF0080E58EC2AF0060E58EC2AF0D1
:108B60001200440E58EC2AF0640E58EC2AF0540E11
:108B700058EC2AF04C0E58EC2AF0440E58EC2AF02F
:108B80001200870E58EC2AF0EB0E58EC2AF0ED0E8E
:108B900058EC2AF0EB0E58EC2AF0870E58EC2AF02D
:108BA0001200810E58EC2AF0B50E58EC2AF0B50EE2
:108BB00058EC2AF0B50E58EC2AF0CB0E58EC2AF0FF
:108BC0001200C30E58EC2AF0BD0E58EC2AF0BD0E70
:108BD00058EC2AF0BD0E58EC2AF0DB0E58EC2AF0C7
:108BE0001200810E58EC2AF0BD0E58EC2AF0BD0E92
:108BF00058EC2AF0BD0E58EC2AF0C30E58EC2AF0BF
:108C00001200810E58EC2AF0B50E58EC2AF0B50E81
:108C100058EC2AF0B50E58EC2AF0BD0E58EC2AF0AC
:108C20001200810E58EC2AF0F50E58EC2AF0F50EE1
:108C300058EC2AF0F50E58EC2AF0FD0E58EC2AF00C
:108C40001200C30E58EC2AF0BD0E58EC2AF0BD0EEF
:108C500058EC2AF0AD0E58EC2AF0CB0E58EC2AF066
:108C60001200810E58EC2AF0F70E58EC2AF0F70E9D
:108C700058EC2AF0F70E58EC2AF0810E58EC2AF046
:108C80001200FF0E58EC2AF0BD0E58EC2AF0810EAF
:108C900058EC2AF0BD0E58EC2AF0FF0E58EC2AF0E2
:108CA0001200CF0E58EC2AF0BF0E58EC2AF0BF0E7F
:108CB00058EC2AF0BF0E58EC2AF0C10E58EC2AF0FE
:108CC0001200810E58EC2AF0EF0E58EC2AF0F70E45
:108CD00058EC2AF0EB0E58EC2AF09D0E58EC2AF0D6
:108CE0001200810E58EC2AF0BF0E58EC2AF0BF0E8D
:108CF00058EC2AF0BF0E58EC2AF0BF0E58EC2AF0C0
:108D00001200810E58EC2AF0FB0E58EC2AF0F70EF8
:108D100058EC2AF0FB0E58EC2AF0810E58EC2AF0A1
:108D20001200810E58EC2AF0FB0E58EC2AF0E70EE8
:108D300058EC2AF0DF0E58EC2AF0810E58EC2AF09D
:108D40001200C30E58EC2AF0BD0E58EC2AF0BD0EEE
:108D500058EC2AF0BD0E58EC2AF0C30E58EC2AF05D
:108D60001200810E58EC2AF0ED0E58EC2AF0ED0EB0
:108D700058EC2AF0ED0E58EC2AF0F30E58EC2AF0DD
:108D80001200C30E58EC2AF0BD0E58EC2AF0AD0EBE
:108D900058EC2AF0DD0E58EC2AF0A30E58EC2AF01D
:108DA0001200810E58EC2AF0ED0E58EC2AF0ED0E70
:108DB00058EC2AF0ED0E58EC2AF0930E58EC2AF0FD
:108DC0001200BB0E58EC2AF0B50E58EC2AF0B50E86
:108DD00058EC2AF0B50E58EC2AF0CD0E58EC2AF0DB
:108DE0001200FD0E58EC2AF0FD0E58EC2AF0810E10
:108DF00058EC2AF0FD0E58EC2AF0FD0E58EC2AF043
:108E00001200C10E58EC2AF0BF0E58EC2AF0BF0E2B
:108E100058EC2AF0BF0E58EC2AF0C10E58EC2AF09C
:108E20001200F90E58EC2AF0E70E58EC2AF09F0ECB
:108E300058EC2AF0E70E58EC2AF0F90E58EC2AF01C
:108E40001200810E58EC2AF0DF0E58EC2AF0EF0EDB
:108E500058EC2AF0DF0E58EC2AF0810E58EC2AF07C
:108E60001200B90E58EC2AF0D70E58EC2AF0EF0E8B
:108E700058EC2AF0D70E58EC2AF0B90E58EC2AF02C
:108E80001200F90E58EC2AF0F70E58EC2AF08F0E6B
:108E900058EC2AF0F70E58EC2AF0F90E58EC2AF0AC
:108EA0001200000E58EC2AF0000E58EC2AF0040EC6
:108EB00058EC2AF00A0E58EC2AF0040E58EC2AF06E
:108EC0001200000E58EC2AF0000E58EC2AF0000EAA
:108ED00058EC2AF0000E58EC2AF0000E58EC2AF05C
:108EE0001200FF0E58EC2AF0FF0E58EC2AF0FF0E8D
:108EF00058EC2AF0FF0E58EC2AF0FF0E58EC2AF03E
:108F00001200280E58EC2AF01200FE0E58EC2AF03F
:108F1000FE0E58EC2AF0000E58EC2AF01200000E5B
:108F200058EC2AF0000E58EC2AF0000E58EC2AF00B
:108F30001200000EAA6E000EA96E1150A86EA69E19
:108F4000A69CA684550EA76EAA0EA76EA682A6B2F0
:108F5000A7EF47F0A6941200000EAA6E010EA96EAC
:108F60001250A86EA69EA69CA684550EA76EAA0EA9
:108F7000A76EA682A6B2BAEF47F0A6941200000E22
:108F8000AA6E020EA96E1350A86EA69EA69CA68479
:108F9000550EA76EAA0EA76EA682A6B2CDEF47F019
:108FA000A6941200000EAA6E030EA96E1450A86EAD
:108FB000A69EA69CA684550EA76EAA0EA76EA68294
:108FC000A6B2E0EF47F0A6941200000EAA6E040EBF
:108FD000A96E1550A86EA69EA69CA684550EA76ED7
:108FE000AA0EA76EA682A6B2F3EF47F0A6941200CF
:108FF000000EAA6E050EA96E1650A86EA69EA69C1F
:10900000A684550EA76EAA0EA76EA682A6B206EF7C
:1090100048F0A6941200000EAA6E060EA96E175014
:10902000A86EA69EA69CA684550EA76EAA0EA76E35
:10903000A682A6B219EF48F0A6941200000EAA6EFE
:10904000070EA96E1850A86EA69EA69CA684550E63
:10905000A76EAA0EA76EA682A6B22CEF48F0A69421
:109060001200000EAA6E080EA96E1950A86EA69ED8
:10907000A69CA684550EA76EAA0EA76EA682A6B2BF
:109080003FEF48F0A6941200000EAA6E090EA96EDA
:109090001A50A86EA69EA69CA684550EA76EAA0E70
:1090A000A76EA682A6B252EF48F0A6941200000E58
:1090B000AA6E0A0EA96E4C9E4C50A86EA69EA69C47
:1090C000A684550EA76EAA0EA76EA682A6B266EF5C
:0690D00048F0A694120016
:020000040030CA
:03000100331800B1
:02000500358044
:060008000FC00FE00F40E5
:0200000400F00A
:0C00000008044BBB9B887F7F00000000C1
:00000001FF
